:100000003DC435C436C4189535C4189534C4189504
:1000100033C41895FFFFFFFFFFFFFFFFFFFFFFFF48
:10002000FFFFFFFFFFFFFFFFFFFFFFFFFFFFFFFFE0
:10003000FFFFFFFFFFFFFFFFFFFF18950C94E50494
:10004000FFFFFFFFFFFFFFFFFFFFFFFFFFFF189511
:100050001CC5FFFFFFFFFFFFFFFF1895B6C4FFFFA2
:100060009DC4FFFFFFFFFFFFFFFFFFFFFFFFFFFF3D
:10007000FFFFFFFFFFFFFFFFFFFFFFFFFFFFFFFF90
:10008000FFFFFFFFFFFFFFFFFFFF1895C2C4FFFF49
:100090003EC5FFFFFFFFFFFFFFFFFFFFFFFFFFFF6B
:1000A000FFFFFFFFFFFFFFFFFFFFFFFFFFFFFFFF60
:1000B000FFFF18950DC51895FFFFFFFFFFFFFFFF1E
:1000C000FFFFFFFFFFFFFFFF48C518957FC418958E
:1000D000FFFFFFFFFFFF18959BC4FFFFFFFFFFFF20
:1000E0001895EEEBFFE90E943401A0938F03B093C3
:1000F0009003009127031091280320916102309111
:1001000062020217130718F40027112702C0021B0E
:10011000130BA8E6B4E00E948001E8E6F4E00E9438
:100120008A0100910E0410910F04202F212B69F4F5
:100130000DEB0093760405E6009377040FEB009334
:10014000780402E300937F0408C0A9E7B4E00E94AA
:100150008001E9E7F4E00E948A010E944C010895C1
:10016000EEE9FFE981D00091DE021127A6E6B4E0B6
:100170000E946B01E6E6F4E08FD00895EEE3FFE91C
:1001800073D0009152031127ACE7B4E00E948001C4
:10019000ECE7F4E00E948A017FD00895EEE1F0EAF6
:1001A0000E9434010091DE021127A0938F03B093C7
:1001B0009003A7E6B4E00E948001E7E6F4E00E9425
:1001C0008A0120916102309162020091270310910F
:1001D0002803021B130BAAE7B4E00E948001EAE7A0
:1001E000F4E00E948A010E944C01A092D20308957B
:1001F000429A0E94FB20449A000002B90E94FB2010
:1002000044980895006801D0089542980E94FB2008
:10021000449A000002B90E94FB204498000008950F
:100220000027F0DF429AB090DF0200E30B29E0DF05
:1002300008950091A9030F3061F00F3441F00F31A0
:1002400021F00F3541F4002706C00FE404C00FE091
:1002500002C00FE300C003950093A903D3DF429AC5
:100260000091A603C5DF0895A0938F03B093900378
:10027000A0E6B4E010E205910D931A95E1F7A09184
:100280008F03B09190030895BDDF429A14E001916D
:10029000AFDF1A95E1F70895E0E6F4E00027B2DF5A
:1002A00010E10191A5DF1A95E1F70E94FB2000E41F
:1002B000A9DF0E94FB2010E101919ADF1A95E1F776
:1002C000089540E3122F12951F70140F1D932F7085
:1002D000240F2D93089511270E9446210E94610149
:1002E00008950091760310917703ACE6B4E00E9484
:1002F0008001ECE6F4E00E948A010E944C0108951E
:100300000E944621F22E232F0E9461012F2D0E9470
:10031000610108950081003339F400E20193008106
:10032000003311F400E201930895EEE7FFE99CDF4A
:10033000009176031127A7E7B4E00E946B01E7E77D
:10034000F4E0AADF0895E2EBF2EA8EDFA5DF0E9477
:1003500009210E94D9205092A9026092AA027092AB
:10036000AB028092AC0208950DEB0D9305E60D9360
:100370000FEB0D9300E20D930D930D930D930895E4
:10038000E2EDF2EA71DF0091E20200FF04C0A7E6AD
:10039000B4E0EADF0AC00091F0071091F107A7E688
:1003A000B4E0AEDFE7E6F4E0B5DF0091E20201FF82
:1003B00004C0A7E7B4E0D8DF0AC00091F2071091AB
:1003C000F307A7E7B4E09CDFE7E7F4E0A3DF64DF2F
:1003D0000E9409210E94D9205092A9026092AA028B
:1003E0007092AB028092AC020895EEE1FFE90E94A8
:1003F00034010E944C01089506B51091BD03011B04
:1004000010F041F52AC01091BE03139509F5209113
:10041000BF032395D9F43091C003339519F43327E2
:10042000222711273093C00368E25BE34EEA003CC9
:1004300014072507360750F033272227112730935A
:10044000C003009132030064009332032093BF0382
:100450001093BE0306B50093BD0308957FEF739517
:100460000050114E254F3540D0F700501F412A4013
:100470003A4F5FEE505F0058164928493040D0F798
:100480000058194627463F4F5395005412442F40B9
:10049000D8F7005C1D4B204F4FEE405F005A1648C6
:1004A0002140D8F7005619472E4F43950051174267
:1004B0002040D8F7005F184D2F4F6FEE605F085E49
:1004C0001340E0F708511C4F639504561040E0F7C5
:1004D0000C5930EF305F0A50E8F7065F300F08958F
:1004E00008950091CE000091CE000091CE000091C1
:1004F000C80005FFFCCF6093CE000E9409210E9436
:10050000D9205092C5026092C6027092C7028092B2
:10051000C8020091CE000091CE000E94FB200E94F4
:1005200009215090C5026090C6027090C702809069
:10053000C80219E02DE330E00E94E82040F001E01D
:1005400011C000916702006400936702E6CF00913A
:10055000C80007FFE2CF0091CE001091C9000F152F
:1005600081F7002708950091ED0403FF11C008E012
:1005700000930F0C0E94D6268827803049F07727F9
:100580000E94A91C05E00093DF02A0922A037CC010
:100590000091E60401FF45C000919002003309F488
:1005A00040C0A0922A03EEE3FEE91EE00E94884EBE
:1005B0006FE00E94894E1091CE001091CE001091F4
:1005C000CE000033C1F010916702106810936702EB
:1005D00010915303116010935303402FEEEDFEE989
:1005E00043DE042F1127ACE7B4E08ADEECE7F4E049
:1005F00091DE52DE0AC0009153030E7F0093530335
:10060000109131031260109331030E946D1F0E94FC
:100610006D1F0E946D1F1091CE001091CE001091A1
:10062000CE000091E60400FD07C0D7D0F09204048C
:100630000F2D0832E0F028C00E9409215090C50219
:100640006090C6027090C7028090C8021CE12EE440
:100650003EE00E94E82088F40E94624700912B034C
:10066000013050F3009167020F7700936702009109
:10067000E60404FF09C052D507C000E800933B031D
:1006800010916702012B17E00895F999FECF0E949F
:10069000D503019331504A09C1F70895F99964C00F
:1006A000ECE4F4E03EE001911191012B3A95E1F781
:1006B000003009F459C031E0E1E6F2E011E01090B9
:1006C0004C04A11421F05AD010924C044DC0E9E61C
:1006D000F2E019E010904D04A11421F04FD01092D7
:1006E0004D0442C0E1E7F2E011E110904E04A11484
:1006F00021F044D010924E0437C0E9E7F2E019E14E
:1007000010904F04A11421F039D010924F042CC046
:10071000E1E8F2E011E210905004A11421F02ED093
:100720001092500421C0E9E8F2E019E2109051045F
:10073000A11421F023D01092510416C0E1E9F2E097
:1007400011E310905204A11421F018D01092520419
:100750000BC0E9E9F2E019E310905304A11421F071
:100760000DD01092530400C0089501912322231646
:1007700021F4132620E008D030E80895212CF5DF7D
:100780001395330FD9F7089522BD11BD00BDFA9A14
:10079000F99A0895F999FECF22BD11BD00BDFA9ACC
:1007A000F99A01E0100F2A1D089522BD11BDF89A93
:1007B000F89A00B5139509F423950895F999FECF99
:1007C00020E00E94C40313950895F999FECF0E947A
:1007D000C403139509F423950895A0934803B09397
:1007E0004903E0933703F09338030091ED030030A1
:1007F000A9F11091EE03103089F12091A50320306A
:1008000069F1E0EFF6E0A0E4B8E055276627FF24A1
:100810003191337009F051606395653049F43C9132
:10082000306850FF3C9350FFF3943D915527662765
:100830000A9571F73C91306850FF3C933D915527E4
:1008400066270091ED0345E01A9511F7A091480342
:10085000B0914903E0913703F0913803089530E7F0
:1008600024E011270FEFB1DF3A95E9F708951895C5
:10087000189518951895189518951895F8940FEFE0
:100880000DBF01E20EBF2EE70027EE27FF271591CF
:10089000F21708F002C0010FFACF011704C000E2FE
:1008A00017E022278BDFEE27FF27AA24DEB7ED31E2
:1008B000F00509F4E8ECA192EF3FFD07C1F7A08233
:1008C0001FEF1DBF01E20EBFFDE9ECE305910093B0
:1008D000E60405910093E70405910093E80405916F
:1008E0000093E90405910093EA0405910093EB0459
:1008F00005910093C40305910093C50305910093EE
:10090000A50305910093EC0405910093ED04059176
:100910000093EE040091EC0400FD38C001FD36C0E8
:10092000F999FECF10E0222731E4E0E6F2E0ADDEF7
:100930001FE431E1E1E0F2E0A8DE11E43CE0E3EEA7
:10094000F3E0A3DE0091E60400FD20C010E638ECE1
:10095000E0EFF4E09ADE10E621E038ECE0EFF5E0BD
:1009600094DE10E622E038ECE0EFF6E08EDE10E6F2
:1009700023E03091C403330FE0EFF7E086DE10EBA5
:1009800023E03091C403E0E4F8E07FDE0E94CE066D
:100990000000000000000E942A21FDC0DFB6D092B6
:1009A0001F0CDEB4D092330CD090340CDD0CD092FE
:1009B000340CD0901F0CDFBED090340CD3FE1895B1
:1009C000D0903B0CD0920B0118951895DFB6D092C1
:1009D0001F0CC0931204D0931304C0911804D0913B
:1009E0001904D090D100D1FCC090D100D1FCC092AC
:1009F000ED0BD090D600D992C0931804D09319046F
:100A0000C0911204D0911304D0901F0CDFBE189532
:100A10001895DFB6D0921F0C70FF1BC0DD24DA944E
:100A2000D0929500449909C0449AD090810CD092FC
:100A30009500D0901D04689404C04498D0901E0482
:100A4000E894D0929400D0902104D0F8D092210460
:100A500018C071FF16C0DD24DA94D09295005F991A
:100A600005C05F9AD0901D04689404C05F98D09030
:100A70001E04E894D0929400D0902304D0F8D09231
:100A80002304D0901F0CDFBE1895DFB6D0921F0C48
:100A900072FF1AC0DD24DA94D0928500479909C00C
:100AA000479AD090800CD0928500D0901F04689413
:100AB00004C04798D0902004E894D0928400D0904D
:100AC0002204D0F8D0922204D0901F0CDFBE1895DB
:100AD000DFB6D0921F0C71FF16C0DD24DA94D092DD
:100AE000A500419905C0419AD0905A0C689404C061
:100AF0004198D0905B0CE894D092A400D0905C0C0C
:100B0000D0F8D0925C0CD0901F0CDFBE1895C0902E
:100B1000E604C4FE1895DFB6D0921F0CC0931204F1
:100B2000D0931304C0911604D0911704D090C9003B
:100B3000D1FCC090C900D1FCC092EC0BD090CE008B
:100B4000D992C0931604D0931704C0911204D09187
:100B50001304D0901F0CDFBE1895DFB6D0921F0C87
:100B6000DD24DA94D0922501D0900801C090310C98
:100B7000D6FC05C0DC28D0920801DD2406C0C09454
:100B8000DC20D0920801D090300CD0922401D0907B
:100B90001F0CDFBE189501E01091EC0410FD0AE077
:100BA00010FD789411FD0FEF0093DF02A092350342
:100BB0000091E70200FDCFC00E9409210E94D920C8
:100BC0005092C5026092C6027092C7028092C8021B
:100BD0000E9409215090C5026090C6027090C70221
:100BE0008090C80214E82EE130E00E94E82080F3F3
:100BF0000091E70401FF14C0EEEFFEE935DBA0939E
:100C00008F03B09390030091610210916202A7E7F5
:100C1000B4E00E948001E7E7F4E00E948A013CDB37
:100C20000E9409210E94D9205092C5026092C602FA
:100C30007092C7028092C8020091ED0400FD33C09B
:100C40001091080112600091EA0404FD0E94924E86
:100C500004FD1093080106B510913B03011B0430FD
:100C6000D0F70091EA0404FD0E94934E0E940921EE
:100C70005090C5026090C6027090C7028090C80272
:100C80001DE221E331E00E94E82028F3009187046F
:100C90000E94770A009188040E94770A0091EA0472
:100CA00004FD0E94944E00916302039551F414E0F8
:100CB000009164020395009364020E94DE03009198
:100CC00063020093630213E00E94DE03C8DD0E940A
:100CD0002A2149DC0091EA0404FF0AC00091E604DD
:100CE00000FF06C000000000000021E02093F30B8D
:100CF0000E9409210E94D9205092C5026092C6022A
:100D00007092C7028092C8020E9409215090C502C9
:100D10006090C6027090C7028090C80219E02DE36F
:100D200030E00E94E82080F30E942A210091E7042D
:100D300001FDFBDAA0923503A092DE020E94092198
:100D40000E94D9205092D1026092D2027092D302B6
:100D50008092D40200001ED30E9409214DDB0000C6
:100D6000FACF9DEF0E94944B0091340C04FFF9CF11
:100D70000E94D64BA092340C0091320C2091C000FE
:100D800025FFFCCF0093C6000091330C2091C000DA
:100D900025FFFCCF0093C600E4CF0895AA24A3BE8C
:100DA000A5BE04B70F7B04BFADBA0FEF0093690077
:100DB0000FE000936A00A0926E00A0926F00A092D4
:100DC0007000A0927100A0927200A092730005E0E2
:100DD00005BDA0928100A0929100A092A100A092D6
:100DE000B100A092B00010E810BF10911C04109345
:100DF00066001FEFA1B810B912B92091ED0420FFD1
:100E000002C0A0B8A2B807E004B901EF03B905B960
:100E10000FEF07B906B908B90093E80B00E80AB963
:100E200019B91BB9ADB81CB91EB9A3BA12BB14BB12
:100E30000FEF2091EC0426FD0FE700BB01270FB94F
:100E400001BBA09201010FEF00930001009302018A
:100E50000FEF00930701012700930601009308019B
:100E6000A092040110930301109305010FEF00936A
:100E70000A01A0920901A0920B010FEF0CBBF8949C
:100E800001E00093040C0093840C000F0093050C08
:100E9000000F0093060C000F0093070C000F009347
:100EA000080C000F0093090C02E000930A0C02E00A
:100EB00000930B0C01E0009313030093F60BA09238
:100EC000F70B0093A20300EA0093470303EA0093A1
:100ED0001D0C04E000933003A092080403E000938B
:100EE000C70B01E00093CF0B0093F40B0091E804D3
:100EF00006FFA092CF0BA092400C039500933C03F9
:100F0000A0920D0400E31AE0009316041093170456
:100F100000E21BE000931A0410931B0400ED1AE09A
:100F20000093180410931904CC24DD240FEF0093D0
:100F30001E0400935B0C00932004A092790C009196
:100F4000E8040770B1F0109165021093DB0B01E02B
:100F50000093210400935C0C00932204F3EAE2E77F
:100F6000059100932C0408E20093E90B01E0009343
:100F7000D104A0921903A0922503A092520300E18C
:100F800000933A030091ED0400FF04C00091820237
:100F90000093410C0091E60400FD7AD00091EC042E
:100FA00003FD84D00091EC0406FD80D00091EA049A
:100FB00004FD8AD00091E60400FFB0D211E0A092B7
:100FC000DC0B04FD1093DC0B0091E904037099F035
:100FD000A092210CA092200C00910102109102021B
:100FE000012B10910302012B10910402012B19F423
:100FF00001E00093200C0091E60407FDA1D01091C0
:10100000080110610091E90404FD1093080105FD39
:101010001093080100E40093310C409173004E7F5F
:10102000409373000091ED0403FF04C00E94424B03
:101030000E945C4B0091ED0404FD0E94A62A0091E1
:10104000E70401FF24C00E946D1F0E946D1F01E094
:101050000E9405010E94FB2002E00E9405010E94FF
:10106000FB2006E00E9405010E94FB200CE0CDD889
:101070000E94FB2008E0C9D80E94FB200AE30E94DE
:1010800005010E94FB200FE0C0D80E94FB200895BC
:1010900008E10093C10003E30093C400A092C000E4
:1010A00006E00093C200A092C500089508E10093F5
:1010B000310103E300933401A092300106E0009374
:1010C0003201A0923501089508E10093D10007E6AE
:1010D0000093D400A092D00006E00093D200A0922A
:1010E000D500089508E10093310103E30093340132
:1010F000A092300106E000933201A09235010895DC
:101100000DE10093C90003E30093CC00A092C80056
:1011100006E00093CA00A092CD0008950DE100936F
:10112000C90007E60093CC00A092C80006E0009337
:10113000CA00A092CD0003E00093D60378940895EE
:10114000A092340C01E00DBD01ED0CBD00000AE0E1
:1011500000933B0C00930B019BDF0E9409210E942E
:10116000D9205092B9026092BA027092BB0280926A
:10117000BC02789408950091ED0400FF10C0959989
:101180001BC000E214E10E94DF21153008F052C0BC
:1011900000E214E10E94DF211530D0F317C0009166
:1011A000E70407FD47C04B9907C008E014E10E941F
:1011B000B121153028F03EC001E0009344033AC04D
:1011C00008E014E10E94B1211530D0F30091DF0254
:1011D000013019F0053009F025C0A092DE020EE0C2
:1011E0000093DF020E9409210E94D9205092A90297
:1011F0006092AA027092AB028092AC0221E020932E
:10120000F30B00E200933A0306ED00932503A0924E
:101210001903A0925203A0922C03A0923903A0922A
:101220002E0308C00E3031F41091440301E010FD8C
:10123000009362030895312E12E3412E222410916F
:101240000601132109F023944A94C9F7122D089539
:101250000091E70200FD10C00E943D090E943D0977
:101260000E943D090E943D090E943D090E943D09DE
:101270000E943D090E943D0908950FEF009313035A
:101280000E94FB2001E000931303089500912F03B7
:1012900000FF34C00091060120E8022309F448C091
:1012A0005090B1026090B2027090B3028090B4028C
:1012B00018E023E030E00E94E82018F4A0922F0309
:1012C00037C0A0922F0301E0009362030091DF0278
:1012D0000E3099F00EE00093DF022BD000E2009375
:1012E0003A0306ED00932503A0921903A09252033E
:1012F000A0922C0301E00093F30B1AC01091ED04AF
:1013000010FF0091060110FD02B310FF20E810FD50
:1013100020E2022369F401E000932F030E94D92008
:101320005092B1026092B2027092B3028092B40203
:10133000089501E0009362030093CE0BA09279031D
:10134000A0927003A0928003A09235030091E7045D
:1013500001FF06C0EEEFF0EA0E9434010E944C014A
:10136000A0920D0400916102109162020093DD0BC6
:101370001093DE0BECE4F4E005E1A1920A95E9F7A5
:10138000089555270894551F1A95E9F7089512E115
:101390002AE708950091E60404FD0E948E4E009114
:1013A000E904037031F00091EC0407FD00000E9495
:1013B000AE390091E60400FF11C00E94FE49009181
:1013C0002A030D7F11F40E94534600912A030E7FD9
:1013D00029F400913A0305FF0E9462470091E60458
:1013E00001FF0EC00091CF03037051F400912A0356
:1013F0000B7F31F4B091DF02B13011F40E948A4EBC
:1014000000912A03003069F4B6DE0091E70400FF82
:1014100008C000910D0400FD04C00E948C4E0E9483
:101420008D4E00910801000000000091EA0400FDCB
:101430000E94844E0091EA0403FD0E94F54C009145
:10144000EA0404FD0E94954E0091ED0403FF06C0DE
:101450000E947E4A0E949A4A0E945C4BB091DF0231
:10146000B93040F5B13011F458D53FC0B23019F45D
:101470000E945B173AC0B33019F40E94ED1E35C0CC
:10148000B43019F40E94C71C30C0B53011F42ED00E
:101490002CC0B091DF02B83019F40E948F4E25C0E5
:1014A000B73019F40E948B4E20C0B63019F40E9458
:1014B000E3281BC0B131C8F4BE3019F40E947B2B65
:1014C00014C0BA3019F40E94904E0FC0B93009F41C
:1014D0000CC0BB3011F40E94984EBC3011F40E9435
:1014E0009B4EBD3011F40E946F2108950895109114
:1014F000E60410FF12C01091C00015FFF8CF009352
:10150000C6000E9409210E94D9205092D102609207
:10151000D2027092D3028092D40208950091810287
:101520001127222704FF07C03091870240916802EB
:10153000349F102D212D03FF06C03AE04091850213
:10154000349F100D211D02FF06C035E0409184023A
:10155000349F100D211D01FF06C032E0409183022F
:10156000349F100D211D00FF04C040918202140F12
:101570002A1D3091890240918A023117420710F4E6
:10158000132F2C2D10930E0420930F04089544273D
:10159000B22EB32A71F0103021F4222733274427CA
:1015A00008C0E22EF32E1A9521F02E0D3F1D4A1D84
:1015B000FACF089500912603003009F4E9C0A09302
:1015C0004803B0934903E0933703F09338031AE0DC
:1015D000E0EFF3E0A1921A95E9F7E0EFF6E00A9563
:1015E000E00FFA1D1081212F23702093F803203083
:1015F00009F4C6C06091ED03202E332422270E94F7
:10160000A420022D2394209201041091ED03019F48
:1016100000912603001900930204442755271091D6
:101620000104153020F04091E7035091E8031A952A
:101630002091E5033091E603AADF240F351F2093A4
:10164000FB033093FC031091ED0300910204101B87
:101650002091E3033091E4039ADF2093FD0330935C
:10166000FE03009126030A95E0EFF4E0E00FFA1D77
:10167000A0EFB6E0A00FBA1D4091ED035091020417
:10168000451B439500271127222733275D91619140
:1016900053FD03C0060F1A1D02C0260F3A1D4A95BE
:1016A000A9F74091FD035091FE030217130758F468
:1016B000201B310B4217530718F44427552739F0E4
:1016C000421B530B04C0021B130B400F510F5F71E1
:1016D0004093FD035093FE035093F4034093F503AE
:1016E000F0900104F090ED03409126034A95002705
:1016F000112722273327E0EFF5E0E40FFA1DA0EFD2
:10170000B6E0A40FBA1D5D91619152FD03C0060FB2
:101710001A1D02C0260F3A1D4F19FA9461F7409125
:10172000FB035091FC030217130758F4201B310BE5
:101730004217530718F44427552739F0421B530B1F
:1017400004C0021B130B400F510F5F734093FB0348
:101750005093FC035093F2034093F3030091F8037A
:1017600001FD05C00091E9031091EA0304C0009156
:10177000EB031091EC0310621093F0030093F1035C
:10178000A0914803B0914903E0913703F0913803E9
:1017900008950091F00324E010E117D80091F103BF
:1017A00014D80091F20311D80091F3030ED80091E0
:1017B000F4030BD80091F50308D808956091010453
:1017C0006A95669561FF03C060FF660F01C063956F
:1017D0000895F4DF95DC606A20EC0AEAF02E0E949E
:1017E000710200FF02C010E24EC0E4DEE093370356
:1017F000F093380306E0E0EFF3E00091C80005FF46
:10180000FCCF000041914093CE000A95B1F7C1DFB3
:101810000E9409210E94D9205092C5026092C602FE
:101820007092C7028092C8020E94FB200E94092188
:101830005090C5026090C6027090C7028090C802A6
:1018400019E02DE330E00E94E82010F011E01BC009
:101850000091C80007FFE8CF0091CE001091C900A9
:101860000A3A11F70E9409210E94D9205092A90238
:101870006092AA027092AB028092AC02E0913703B0
:10188000F09138031127089501E00093CF0302E09F
:101890000093CD0308950091CF0304600093CF031C
:1018A000089514E122244A9923941A95E1F7122D00
:1018B000089514E122241C9923941A95E1F7122D1E
:1018C00008952091DE0220FDF4DF21FDEADF1231D0
:1018D00010F4112706C02091DE0220FD10E121FD49
:1018E00014E01093AF0308950895003009F01395A4
:1018F0000895089500914C0410914D04012B10910E
:101900004E04012B10914F04012B089512951F7066
:101910000895F89410E1109335032091C20B2F73B2
:101920001091C30B1093330420933404A092370416
:10193000A092200CA0923C0C2091C40B2F7110910E
:10194000C50B10932D0420932E040AE50E94770AFC
:1019500008E000932A037093D00B0895F894209127
:10196000C20B2F731091C30B10930102209302023C
:101970002091C40B2F711091C50B1093030220937B
:1019800004020E94D14204E00093DF0201E00093D0
:1019900035030AE50E94770A08E000932A03709352
:1019A000D00B7894089599270091CF0B00FD5EC06D
:1019B00080FD0E94752F01B3026001BB0E940921C6
:1019C0000E94D9205092D60B6092D70B7092D80B00
:1019D0008092D90B0E9409215090D60B6090D70BB2
:1019E0007090D80B8090D90B14E82EE130E03327AB
:1019F0001091090220910A020091EC0407FD31E0E8
:101A00000E94E82060F580FD13C081FF07C002E05E
:101A100010E20E94B1219927153090F008E010E201
:101A20000E94D521992781FD92E0153048F0D2CF50
:101A300008E010E20E94CC219927153008F0CACFA7
:101A40000091EC0407FD0E948B1F01B30D7F01BBC9
:101A500091FF0CC091E008EE0E94770A07C001B325
:101A60000D7F01BB91E005EE0E94770A892F0E944D
:101A70006D1F0E946D1FA092080108959AE51091B4
:101A8000CF0B10FD3DC080E1602F60FD0E94752FDF
:101A900060FD80E231E001B3032B01BB0E9409210C
:101AA0000E94D9205092D60B6092D70B7092D80B1F
:101AB0008092D90B0E9409215090D60B6090D70BD1
:101AC0007090D80B8090D90B14E82EE130E0109183
:101AD00005022091060296EE0E94E82040F49AE565
:101AE000082F10E20E94C321153008F0E3CF01B3A4
:101AF0000E7F01BB0E946D1F0E946D1FA092080106
:101B000008951091CF0B10FD15C00E94752F54E061
:101B100001B3052B01BB000000000000AEDBADDB14
:101B2000ACDB01B30B7F01BB0E946D1F0E946D1FD8
:101B3000A092080108959AE51091CF0B10FD61C0A5
:101B4000602FA092390321E01091EC0415FD209341
:101B5000390361FDA092390362FDA092390380E14F
:101B600061FD0E94752F61FD80E28093C10354E006
:101B700001B3052B01BB0E946D1F0E9409210E9429
:101B8000D9205092D60B6092D70B7092D80B8092CE
:101B9000D90B9CEC0E9409215090D60B6090D70B7A
:101BA0007090D80B8090D90B14E82EE130E01091A2
:101BB0009F022091A0020E94E820C8F48091C103F6
:101BC0000091390300FF07C001E010E20E94B1213B
:101BD0009AE5153060F0082F10E20E94D5219AE5B1
:101BE0000091390300FD94EE153008F0D2CF01B317
:101BF0000B7F01BB0E946D1F0E946D1FA092080108
:101C0000092F08958827000000000091CF0B00FDE8
:101C10009BC0002733DF9A3559F00091DF020E3068
:101C2000B9F39093230301E029DF909123031DC0B2
:101C300088270E949A3F0091EE0402FF07C082E0CD
:101C4000B2DE80FF03C081E0AEDE12C001E016DF2D
:101C50009A3509F00AC000276EDF9A35D9F09093C3
:101C6000230302E068DF90912303092F0E94770A83
:101C70000091DF020E3061F200912A03077F00938A
:101C80002A0301E00093DF02A0923503A092C00B6B
:101C900081E05AC001B3006401BB0E946D1F02E0E5
:101CA0004ADF9A3521F001B30F7B01BBDECF00275D
:101CB000E5DE9A3559F00091DF020E3051F3909332
:101CC000230301E0DBDE90912303EDCF0091EE04CE
:101CD00002FF04C001B30F7B01BB1DC084E00E9462
:101CE0009A3F01E0CBDE9A3509F0DDCF04E023DF37
:101CF0009A3551F09093230301B30F7B01BB02E0AF
:101D00001ADF90912303B1CF01B30F7B01BB02E037
:101D100012DF9A3501F00091EE0402FF0EC081E05F
:101D200042DE80FDA5CF84E00E949A3F01E0A6DE5E
:101D30009A3509F09DCF882707C088270091740C39
:101D400000FF02C081E02FDE089588270000000018
:101D50000091CF0B00FD73C0002790DE9A3559F03B
:101D60000091DF020E30B9F39093230301E086DE89
:101D70009091230337C00091EE0405FF09C082E073
:101D800012DE80FF05C081E00EDE01E077DE70CF5D
:101D900088270E949A3F0091EE04047161F082E06E
:101DA00002DE80FF08C081E0FEDD84E00E949A3FF1
:101DB00001E064DE5DCF01E061DE9A3509F012C01A
:101DC0000091EE040670D1F10027B5DE9A35F9F0E6
:101DD0000091DF020E30D1F09093230302E0ABDEDE
:101DE00090912303092F0E94770A0091DF020E30A1
:101DF00069F000912A03077F00932A0301E0009312
:101E0000DF02A0923503A092C00B81E018C081E0F0
:101E1000CADD77DE002732DE9A3559F00091DF0205
:101E20000E3069F09093230301E028DE90912303A4
:101E3000CFCF01E023DE9A3509F0CACF8827089575
:101E40000091CF0B00FD49C00091EE0405FF11C0C9
:101E5000002714DE9A35E1F481E00E94D30C80FD66
:101E600017C08827000001E009DE9A3589F400E2F6
:101E7000A9F104FF24C081E00E94D30C80FD08C0BA
:101E80000027FCDD9A3521F401E0F8DD9A35D9F020
:101E9000092F0E94770A01E0F1DD0091DF020E3088
:101EA00071F100912A03077F00932A0301E0009358
:101EB000DF02A0923503A092C00B81E020C004E0B5
:101EC0003ADE9A3529F701B3086001BB0E946D1F05
:101ED0000E946D1F01B3077F01BB00E10093350332
:101EE0000DE50E94770A0E9409210E94D920509294
:101EF000D60B6092D70B7092D80B8092D90B0895B5
:101F00000091CF0B00FD08C002E015DE0091740CBB
:101F100000FF02C081E047DD08950091EB0402FD5F
:101F200095C60091ED0400FDF4C605FDD9C60091EB
:101F3000EE0406FDD8C60091E60400FF70C60091CD
:101F40003503003009F40FC000FD7CC201FDACC3B5
:101F500002FD23C403FD86C404FD8FC505FD27C60D
:101F6000A09235037EC700912A0300FD7AC7009135
:101F7000C00B007E003209F074C777272224332477
:101F800044248824A092F50B2091C20B0091C30B2E
:101F90003091ED04307921F43091200C30FF0AC0EB
:101FA0003091C20B307C442737FD446036FD4160E0
:101FB00040930C042F73022B59F071601091C30BE6
:101FC0000E948F3F1093C80B2093C90B3093CA0B0C
:101FD0002091C40B0091C50B2F71022B59F0746036
:101FE0001091C50B0E948F3F1093CB0B2093CC0B0D
:101FF0003093CD0BA0923F0C0091ED0401FF0BC07C
:102000000091C00B0F701091C10B012B21F001E06A
:1020100000933F0C8CC00091ED04067909F42CC0AC
:102020001091C10B1F771093740C1091C10B129576
:102030001F701695169516950091C00B0F71000F25
:10204000102B1093730C007302951091EE0412FD87
:1020500000934B041091C40B107E129516951093AB
:10206000210CA092C00B11FF62C010FF52DC109136
:10207000210C10FD73DCF5C60091ED0403FF12C0C6
:102080002091C00B27701091C10B8894110F221F53
:10209000110F221F110F221F110F221F1093770CF7
:1020A0002093780C0091C00B087106950695069553
:1020B00000934B040091E90402FF39C07093220C95
:1020C0002091C00B0091C10B00934B042F70022B89
:1020D00071F10091CE0B00FD0CC00091CF0B00FF01
:1020E00008C020918E022093C00B00918D020093B6
:1020F000C10B0091E90402FF8ECF0091CE0B00FDD1
:1021000072601091C10B0E948F3F10933504209391
:102110003604022F012B59F40091CE0B1091CF0BF6
:10212000012B29F405EC0E94D549F89440C0009198
:10213000CE0B00FF0FC01091C20B107C442717FD7F
:10214000446016FD41601091C00B107114FD426097
:1021500040930C04A092C00B0E942A210091E80435
:1021600006FDDEC00091CE0B00FD8BC00091210C5E
:10217000037009F086C00091E804017069F10E94C3
:102180004D4A203049F106EC009323030091200CC6
:1021900000FD09C020FF1AC081E00E949841009113
:1021A000230307FF0FC0009123030E94770A7727BC
:1021B000A0923503A092C00B00912A03077F0093E1
:1021C0002A034FC60E944D4A203031F00E9411422E
:1021D0000091230307FDE7CF0091E804027041F06E
:1021E0000E94F34A203021F007EC0E94770ADFCFEB
:1021F0000091EC0403FD2BC00091ED0402FD41C0F1
:10220000009108010160009308010E946D1F0E9467
:10221000981EA09208010091E904007851F03091D5
:10222000EA0B3B7F0E946D4A213009F03460309305
:10223000EA0B0091E804087051F03091EA0B377F07
:102240000E941F4B213009F038603093EA0B009157
:10225000ED0403FF08C001E000930F0C0E94D62696
:10226000803009F0C5C10091E804007151F030914F
:10227000EA0B3D7F0E94314B213009F032603093F0
:10228000EA0BA092C00B0E942A210091E70403FFF1
:1022900013C00091F40B00FF0FC0A0923B030E94FB
:1022A000FB2100FFFCCF0E946D1F009108010E7FF3
:1022B00000930801A092F40BA0928B030AE50E9400
:1022C000770A0091200C00FF05C083E00E9458406F
:1022D0007091220C0091EE0401FF1CC000E210E29C
:1022E0000E94D521153038F002E025DC9A3519F02E
:1022F000092FFDD85CCF0E94044B503019F007EC39
:10230000F6D855CF0091740C00FF04C088274BDB32
:1023100080FD4DCF0091210C037011F40E948F437A
:1023200008E000932A037093D00B70FD429872FD71
:10233000459871FD5F980E946D1F0E94CB3E70FD15
:102340000E94403D71FD0E94833D72FD0E94C63D8A
:102350003327442770FD0E94523E71FD0E94703E5B
:1023600072FD0E948B3E70FD3093710071FD5093A1
:10237000720072FD40936F0003E070FD00939100C6
:1023800071FD0093A10072FD009381000091EC04A7
:1023900003FD06C099270091CE0B00FD0E94443F2B
:1023A0000E9409210E94D9205092D60B6092D70B2F
:1023B0007092D80B8092D90B5092DA046092DB04B1
:1023C0007092DC048092DD045092DE046092DF049F
:1023D0007092E0048092E1045092E2046092E3047F
:1023E0007092E4048092E5045092B9026092BA02BD
:1023F0007092BB028092BC0201E000933503009111
:10240000E9040073E1F0002770FD00E272FD006155
:102410000DBBA0920C0CA0920D0CA092000CA092EF
:10242000010CA092FE0BA092FF0BA092160CA092A2
:10243000170CA092140CA092150CA092FD0B78948E
:1024400000000FC5703009F458C00091CF0B00FD9B
:1024500034C00091CE0B00FD30C00091E804017043
:1024600061F10091210C037041F50091DA0B00FD40
:1024700024C00E9409215090D60B6090D70B709019
:10248000D80B8090D90B14E82EE130E00E94E820B0
:1024900008F4E7C401E00093DA0B0E944D4A2030B3
:1024A00061F40E94FD3C0E94E83C71FD0E94123DD7
:1024B000F89408EC0E94D54911C00E94092150905F
:1024C000D60B6090D70B7090D80B8090D90B10ED85
:1024D00022E133E10E94E82008F4C3C40E94FD3CDD
:1024E0000E94E83C71FD0E94123DF89409EC0E94A4
:1024F000770A0E946D1F0C94D710F8940091EE0497
:10250000067331F101FD08C000914B0400FD04C0C9
:102510001CDC80FD12C003C075DB80FD0EC00E9474
:10252000CE2E009325030091EA0B0093520321E085
:102530002093F30B0AEA009319037727A09235033F
:10254000A092C00B00912A03077F00932A0389C43D
:102550000091EC0403FF55C00091ED0404FD29C077
:1025600003FF0CC003E000930F0C0E94D6268030BE
:1025700009F03EC000E10093350373C401EA009303
:10258000D30301E000930F0CA0921C0CA092D60381
:10259000A092130C0E94B22280FFFCCF00E10093B6
:1025A00035030091670200FF5CC40BEC0E94D54923
:1025B000BCC101E000930F0C0E942D248030C1F4B7
:1025C0000E94CE2E009325030091EA0B0093520344
:1025D00021E02093F30B0AEA00931903A092EA0B7F
:1025E000A0920C047727A0923503A0922A0339C445
:1025F00077270E94A91C05E00093DF02A0922A031E
:1026000030C40091CE0B00FDD2CD0091CF0B00FD68
:1026100028C00091E80407FF24C00E9409215090BF
:10262000D60B6090D70B7090D80B8090D90B14EB21
:1026300024EC34E00E94E82008F009C0309910C072
:1026400010E401E00E94E8211A3050F40AC02F98EB
:102650000AEC0E94D5497091D00B45E040930C04E0
:1026600000C40091ED0402FD01C0000002E00093EF
:1026700035030E946D1F0091E90402FF05C09927F0
:1026800072E00E94443FEDC301B3016001BB0E94B0
:1026900009210E94D9205092D60B6092D70B7092DC
:1026A000D80B8092D90BDDC30E9409215090D60B24
:1026B0006090D70B7090D80B8090D90B14E82EE166
:1026C00030E0109105022091060233270E94E82095
:1026D00078F40091E80402FFC4C300E120914B04A8
:1026E00020FD00E212E30E94C321153008F0B9C3B7
:1026F0000091E90402FD03C001B30E7F01BB00910C
:10270000ED0402FD11C001B30D7F01BB0091EE0489
:1027100004FD1EC00E946D1F0E946D1F00910801E4
:1027200001600093080109C00E946D1F0E946D1F87
:10273000009108010160009308010E946D1F0E9432
:102740006D1F0091ED0402FD03C001B3026001BBE7
:1027500088270091EB0404FD0E94CE408827009159
:10276000EB0401FF0E949A3F0091EE0480E004FD1B
:102770001AD904E0009335030E9409210E94D92050
:102780005092D60B6092D70B7092D80B8092D90BD7
:102790000091ED0402FD42C064C30E9409215090E3
:1027A000D60B6090D70B7090D80B8090D90B14E8A3
:1027B0002EE130E01091090220910A0233270E9495
:1027C000E82008F010C00091CF0B00FD14C000916C
:1027D000E804087081F00091EA0B087061F40E942F
:1027E0001F4B213041F00BEC0E94D5490091EA0BC0
:1027F00000610093EA0B0091E90402FF0FC04091D1
:102800000C04426040930C049091600272E00E94BC
:10281000443F08E00093350386FD23C30091EE0496
:1028200004FF0DC00E946D1F0E946D1F00910801E2
:102830000160009308010E946D1F0E946D1F01B38B
:10284000016001BB0E9409210E94D9205092D60B41
:102850006092D70B7092D80B8092D90B08E000934E
:102860003503FFC20091E90402FDE4C00E94092182
:102870005090D60B6090D70B7090D80B8090D90BEE
:1028800014E82EE130E01091050220910602332772
:102890000E94E82058F40091E80402FFE2C200E23E
:1028A00012E30E94D5211530E8F0DBC20091CF0B76
:1028B00000FD18C001B30E7F01BBF8947727A092EA
:1028C000C00B0FEF08B9A09235030E946D1F0E9444
:1028D0006D1F009108010E7F009308010BEC0E9410
:1028E000770ABFC201B30E7F01BB0091ED0402FD68
:1028F000A1C00091EA0B04FF9DC001B30D7F01BB95
:102900000E946D1F0E946D1F009108010E7F0093B1
:1029100008010E946D1F01B3026001BB0E948E1F5F
:102920000E948E1F01B30D7F01BB00913B041091EB
:102930003C0420913D043091E90B030F1A1D2A1D20
:1029400000933B0410933C0420933D040091380411
:102950001091390420913A043091E90B030F1A1DAC
:102960002A1D009338041093390420933A0470917F
:10297000D00B40910C040091200C15E000FF45E0C5
:1029800000FD412740930C040E948342A092C00B9B
:1029900000E2009335030E9409210E94D920509241
:1029A000D60B6092D70B7092D80B8092D90B5092B5
:1029B000DA046092DB047092DC048092DD045092B1
:1029C000DE046092DF047092E0048092E104509291
:1029D000E2046092E3047092E4048092E504509271
:1029E000B9026092BA027092BB028092BC0200915E
:1029F000E9040073E1F0002770FD00E272FD006160
:102A00000DBBA0920C0CA0920D0CA092000CA092F9
:102A1000010CA092FE0BA092FF0BA092160CA092AC
:102A2000170CA092140CA092150CA092FD0B789498
:102A3000000017C20091E90406FF14C000918B0347
:102A400000FD10C014E600E10E94C3211A3050F0CE
:102A50000CEC0E94D5490091CF0B00FF00FF01C292
:102A60000E946D1F0BE50E94D5490091ED0407FD02
:102A7000A7CD00E100933503F4C10091200C00FDC7
:102A8000F1D1A092080177271091330420913404EA
:102A9000022F012B003049F00091370400FF05C0E0
:102AA00000910C04036000930C0471600E948F3F3E
:102AB000109338042093390430933A0410912D0474
:102AC00020912E0440910C0444FD446040930C047A
:102AD00045FF04C03091360C1A0D2A1D022F012B20
:102AE000003049F074600E948F3F10933B042093A4
:102AF0003C0430933D047093D00B703009F402C055
:102B00000E9483420E9409210E94D9205092D60B34
:102B10006092D70B7092D80B8092D90B5092DA0446
:102B20006092DB047092DC048092DD045092DE043B
:102B30006092DF047092E0048092E1045092E2041B
:102B40006092E3047092E4048092E5045092B9022A
:102B50006092BA027092BB028092BC0202E00093C3
:102B6000DF0201E0009335030091E9040073E1F016
:102B7000002770FD00E272FD00610DBBA0920C0CFD
:102B8000A0920D0CA092000CA092010CA092FE0B42
:102B9000A092FF0BA092160CA092170CA092140CFE
:102BA000A092150CA092FD0B789400005AC17030D1
:102BB00011F00C943117F89484E00091200C00FD82
:102BC0000E945840D9D6A0923B030091E70403FF2E
:102BD00007C00E94FB2100FFFCCF01E00093F40B33
:102BE0007CE50091E804037029F00E944D4A2030F2
:102BF00009F079EE072F0E94D54901E00093DF022A
:102C0000A0923503A092C00B00912A03077F009386
:102C10002A03A092EA0BA0920C047727F894009163
:102C2000E70407FF06C00E947C4D0091840C00FF62
:102C30009AC90E9409210E94D9205092A90260924B
:102C4000AA027092AB028092AC020BC10091DE022C
:102C5000003009F406C1033378F59090DE029A94AF
:102C6000E0EBF3EAE90DFA0D049107700BB90E944D
:102C70006D1FE2EEF3EAE90DFA0D049101BB0E942B
:102C80008E1FABB8A1BA0E948E1FE4E1F4EAE90DF1
:102C9000FA0D04910BB90E946D1FE6E4F4EAE90D08
:102CA000FA0D049101BB0E948E1FABB8A1BA00912E
:102CB000DE020E94770AD1C0073309F0CEC000912E
:102CC00008010160009308010E948E1F0E948E1F60
:102CD0000E948E1F009108010E7F00930801BDC065
:102CE0000E94BC1EBAC00091DE02003089F00E9432
:102CF00009210E94D9205092D60B6092D70B709276
:102D0000D80B8092D90B0CE00093DF02A092350320
:102D1000A8C00091DE021091E60B003039F00930B6
:102D200028F4103019F0193008F401C096C07093DF
:102D3000D00BA092F70B00930204109301040091B2
:102D4000E80406FD4AC00E94994E0E946D1F10E2E1
:102D500004E00E94B121009172000E7F0093720086
:102D6000153040F001E00093F70B0EE50E94770A62
:102D70000E946D1F009108010160009308010E94EC
:102D80006D1F009108010860009308010E946D1FEB
:102D900000910801077F009308010E946D1FA09217
:102DA000080110E208E00E94CC21153020F007EC69
:102DB0000E94770A45C010E208E00E94B121153058
:102DC00020F006EC0E94770A3BC00E94964E10FD50
:102DD00004C005EC0E94770A33C0009102041091F0
:102DE000410CA0923C03011760F0009108010160C2
:102DF0000093080100933C030E946D1F0EE50E94A2
:102E0000770A009108010260009308010BE000932B
:102E1000DF02A09235030E9409210E94D92050921E
:102E2000D60B6092D70B7092D80B8092D90B509230
:102E3000C9026092CA027092CB028092CC020DC08D
:102E400000912A03077F00932A03A09202040091B5
:102E50003A031EE004FF1093DF02A092DE02A0926C
:102E6000E60B08950091C20B0F731091C30B22273C
:102E70003091EB0434FD2091E50312170A0518F494
:102E80001127002702C0121B0A0910933304009374
:102E900034040091C40B1091C50B10932D040093C2
:102EA0002E04A092370440910C0442FF40614B7FF6
:102EB00040930C0408950091E60400FF48C500917A
:102EC000350300FD0FC001FDF7C002FDB6C103FDD3
:102ED00053C204FD9AC205FDA4C306FD77C407FDD5
:102EE000AAC406C5703059F10E9409215090D60B32
:102EF0006090D70B7090D80B8090D90B10ED22E129
:102F000033E10E94E82008F423C5F8940E94FD3CB8
:102F10000E94E83CA0923503A092C00B71FD0E9474
:102F2000123D77270DEC0E94770A00912A03077F54
:102F300000932A0305E00093DF020C94A81CF89488
:102F40000091ED0401FD5AC30091ED0404FD4DC054
:102F500003FD20C088270091200C00FD84E00E9422
:102F600058400091CF0B00FD15C00091E80400719E
:102F700089F00091EA0B01FD0DC00E94314B203019
:102F800049F0009167020062009367020EEC0E9414
:102F9000D549F3C20091EC0403FF51C00091ED0448
:102FA00004FD23C003FF09C006E000930F0C0E943C
:102FB000D626803009F03BC022C002EA0093D3033A
:102FC00001E000930F0CA0921C0CA092D603A092DB
:102FD000130C0E94B22280FFFCCF0091670200FF19
:102FE000CCC20FEC0E94D549C8C288270E94584025
:102FF0000BE000930F0C0E942D248030C1F4A092AE
:1030000008010E946D1F94D60DE50E94770A0E9468
:1030100009210E94D9205092D60B6092D70B709252
:10302000D80B8092D90B00E10093350391C4772728
:1030300090D405E00093DF02A0922A0389C4009196
:10304000EE0400FDDCCF0091E90402FD26C00091F2
:10305000EE04067339F00E94200F0091EB0406FD88
:1030600029C376C40091ED0402FF06C00091080157
:103070000E7F009308010BC001B30D7F01BB2DD75C
:103080000E946D1F009108010E7F0093080125D753
:103090000E946D1F01B3016001BB0E9409210E94C3
:1030A000D9205092D60B6092D70B7092D80B809299
:1030B000D90B02E0009335030091E80407FF5CC0E0
:1030C0000091CF0B00FD1BC00091D1021091D202E4
:1030D0002091D40250166106720608F009C0309B98
:1030E0000DC010E401E00E94E821123338F007C05F
:1030F0002F9A0AED0E94D5490E94BC1C29C42F9A20
:103100000091CF0B00FD11C000918B030F7A00934B
:103110008B0314E601E00E94C3211A3030F00091C5
:103120008B03006100938B0318C00091CF0B00FD4F
:1031300014C00E946D1F14E601E00E94C3211233E7
:1031400060F400918B03006100938B0306C00BEDCC
:103150000E94D5490E94BC1CFBC30091050210913E
:10316000060222270093D1021093D2022093D402A8
:1031700004E000933503ECC30091E90402FD5DC057
:103180000E9409215090D60B6090D70B7090D80BFD
:103190008090D90B1EE027E237E0109105022091C4
:1031A000060233270E94E82058F40091E80402FF49
:1031B000CFC300E112E30E94C321153010F1C8C350
:1031C0000091CF0B00FD1DC001B30E7F01BBF89431
:1031D0007727A092C00B0FEF08B9A092350305E046
:1031E0000093DF02A0922A030E946D1F0E946D1FB0
:1031F000009108010E7F009308010BEC0E94770AF2
:10320000A7C301B30E7F01BB04E000933503009117
:10321000ED0402FF01C061C060D601B3026001BBD2
:103220000E9409210E94D9205092D60B6092D70BA0
:103230007092D80B8092D90B8BC304E000933503B6
:103240000091E80407FF0C9447190091D1021091F6
:10325000D2022091D40250166106720608F00CC00A
:103260000091CF0B00FD74C310E401E00E94C32164
:103270001A3008F06DC30BC00091CF0B00FD07C0E2
:1032800006C001EE0E94D5490E94BC1C61C300919A
:10329000E90402FD50C00E9409215090D60B6090B5
:1032A000D70B7090D80B8090D90B1EE027E237E047
:1032B0001091090220910A0233270E94E82008F4A5
:1032C00047C301B30D7F01BB08D60E946D1F00915B
:1032D000080101600093080100D655270091EB0416
:1032E00006FF02C051E00BC00091ED0402FF07C0D1
:1032F00000910801016000930801EFD551E01091A1
:10330000660222270091200C00FF0E94F43FF894EF
:1033100001B3016001BB00E1009335030E94092164
:103320000E94D9205092D60B6092D70B7092D80B86
:103330008092D90B0DC340910C044D7F40930C0437
:1033400072E0992710910D0220910E020E948F3F8A
:1033500010933504209336040E94443FBED5BDD55A
:10336000EDE1FF2700910B020093D10200910C02C6
:103370000093D202A092D4020E9409215090D60B51
:103380006090D70B7090D80B8090D90B1EE027E28D
:1033900037E00E94E82008F4DBC240910C04426050
:1033A00040930C0472E0909160020E94443F86FDBD
:1033B000CFC200918B030F7E00938B030091CF0B44
:1033C00000FD17C00E946D1F14E601E00E94C3219A
:1033D000123378F400918B03006100938B0309C0D2
:1033E00002EE0E94D5490091CF0B00FF0E94BC1C49
:1033F000AFC20E9409210E94D9205092D60B609240
:10340000D70B7092D80B8092D90B0091ED040879FC
:1034100009F44AC00091E80406FD06C00E94044B6E
:1034200051FD26C050FF94C20E948E1F0E948E1F25
:103430000E948E1F0E948E1F0E948E1F0E948E1F50
:103440000E948E1F0E948E1F0E948E1F0E948E1F40
:103450000E9409210E94D9205092D60B6092D70B6E
:103460007092D80B8092D90B00E20093350370C2A2
:10347000009108010160009308015AD409EC0E94F0
:10348000770A01E00093DF02A0923503A092C00BFF
:1034900000912A03077F00932A03A092EA0BA092CF
:1034A0000C047727F89454C20091E80407FF0C94A9
:1034B0008F1A0E9409215090D60B6090D70B709004
:1034C000D80B8090D90B1EE027E237E00E94E8205D
:1034D0001091050220910602332708F008C010E47D
:1034E00001E00E94C3211A3008F032C212C00091DC
:1034F000CF0B00FD0EC0000000918B030061009314
:103500008B0307C003EE0E94D5490091CF0B00FF4B
:103510001CC200918B030F7E00938B032EC0009181
:10352000ED04087151F50E9409215090D60B60906E
:10353000D70B7090D80B8090D90B1EE027E237E0B4
:10354000109105022091060233270E94E82050F4D2
:103550000091E80402FFFCC100E212E326D7153017
:1035600008F0F6C101B30E7F01BBB7D40E946D1FF6
:10357000009108010E7F009308010091670201721B
:1035800009F01BC00091CF0B00FD14C00091E904AD
:1035900007FF10C03091EA0B32FF0CC00E946D4A49
:1035A000203041F004EE0E94D5493091EA0B34609E
:1035B0003093EA0B0DE50E94770A81E00091200C20
:1035C00000FF0E945840A0923003A092D00B3324F9
:1035D0004424882499241127662777270091200CFA
:1035E00000FD0AC00E94D142789404E00093DF02FB
:1035F00001E000933503ACC10BD2AAC101B3046052
:1036000001BB00E2009335030E9409210E94D920EA
:103610005092D60B6092D70B7092D80B8092D90B38
:1036200097C10091ED04087909F46CC00091E80499
:1036300006FD06C00E94044B51FD62C050FD88C1CA
:103640000091ED0407FF0FC00E94752F0E94981E85
:103650000E946D1FA09208010091EE04067011F007
:103660000E94800F27C004FD0BC003FF4BC00E94C7
:10367000752F0E94981E0E946D1FA0920801B2CF64
:103680000E94752F0E94981EA09208010091E804E4
:1036900006FD09C010E400E40E94D5211A3018F09C
:1036A0000E94981E55C10CE000930F0C0E942D241F
:1036B0008030F1F481E00E94584001E00093DF0285
:1036C000A0923503A0922A030E94CE2E00932503D8
:1036D0000091EA0B0093520321E02093F30B0AEAD6
:1036E00000931903A092EA0BA0920C04772730C133
:1036F0000E94A91C05E00093DF02A0922A0328C1C2
:1037000007ECBDCE0E9409215090D60B6090D70BDC
:103710007090D80B8090D90B14E82EE130E0109116
:103720000702209108020E94E82050F500E112E310
:103730003CD6153008F00CC101B30B7F01BB5527F7
:103740001091E3032091E4030E94F43F00913F0CA9
:10375000003029F101B3016001BB06E00093DF02F4
:1037600001E0009335030E9409210E94D920509264
:10377000D60B6092D70B7092D80B8092D90BE8C011
:103780000AEC0E94770A0091E80406FDD5CF05E017
:103790000093DF02A0923503A0922A03D9C001B39F
:1037A000006201BB9AD301B30F7D01BB00E400931B
:1037B00035030E9409210E94D9205092D60B6092B5
:1037C000D70B7092D80B8092D90BC2C00E940921EE
:1037D0005090D60B6090D70B7090D80B8090D90B7F
:1037E00017E823E933E00E94E820B0F400E412E394
:1037F000DCD5153008F4ACC000E8009335030E9416
:1038000009210E94D9205092D60B6092D70B70925A
:10381000D80B8092D90B9CC00AEC0E94770A0091C9
:10382000E80406FDE9CF05E00093DF02A09235032E
:10383000A0922A038DC00E9409215090D60B60905F
:10384000D70B7090D80B8090D90B17E823E933E0A1
:103850000E94E82050F40091400C00FD79C000E483
:1038600012E3A3D5153080F073C00AEC0E94770AEA
:103870000091E80406FD08C005E00093DF02A09275
:103880003503A0922A0364C00091080101600093EF
:10389000080123D30E946D1F01B3006201BB0E9487
:1038A0006D1F01B30F7D01BB0E946D1F0E946D1F34
:1038B000A092080151E01091E3032091E4030E94DB
:1038C000F43F0091080101600093080106D301B3A1
:1038D000046001BBA09235030E9409210E94D920F7
:1038E0005092D60B6092D70B7092D80B8092D90B66
:1038F0000E9409215090D60B6090D70B7090D80B86
:103900008090D90B14E82EE130E01091070220914D
:1039100008020E94E82030F400E212E346D5153098
:1039200080F016C00AEC0E94770A0091E80406FDB8
:1039300008C005E00093DF02A0923503A0922A039D
:1039400007C00E94D142789450CE0E94BC1C000057
:1039500008950CEC0E94770A082F000F000F000F4B
:10396000000F000F1091750C012B0E94770A009137
:103970000F0C0E94770A0895A092C00B00912A03B1
:10398000077F00932A038091E80B88B9089500917E
:10399000350300FD0DC001FDC0C002FDE8C003FD00
:1039A00082C104FD93C105FD40C1A0923503BFC192
:1039B000703071F10E9409215090D60B6090D70BA6
:1039C0007090D80B8090D90B1CE12EE43EE00E9451
:1039D000E82008F4ACC1F8940E94FD3C0E94E83C49
:1039E00071FD0E94123D77278827A092350305E0DC
:1039F0000093DF02A092C00B00912A03077F00937F
:103A00002A030FEC0E94770A0E946D1F0C94971EE8
:103A1000F8940091EC0410910801127803FF1093C0
:103A2000080101B3007C01BB0091E80B08B98CE5EB
:103A3000809323030091E804017011F10E948E1F0E
:103A40000E944D4A2030E1F006EC009323030091E0
:103A5000200C00FD09C020FF0DC081E00E949841AC
:103A60000091230307FF02C077270AC00E944D4A36
:103A7000203031F00E9411420091230307FDF4CF62
:103A80008091230387FF07C00091200C00FD03C035
:103A900081E00E942841009123030E94770A772742
:103AA00088270091ED0403FD0CC00091E70403FD9D
:103AB0002EC00091EE04047121F40091E80401FD90
:103AC00032C001E00093DF02A0923503A092C00B48
:103AD00000912A03077F00932A0300916702017275
:103AE00009F025C1F8940E94CE2E00932503009181
:103AF000EA0B0093520321E02093F30B0AEA0093B0
:103B00001903A092EA0BA0920C04772710C102E0DF
:103B100000933503A0923B030AC16DD400FF07C197
:103B200001E00093F40B04E0009335030091E804F6
:103B300006FD0CC001FF0BC000E414E636D41830BB
:103B400028F00091EA0B00620093EA0BF1D00EE539
:103B50000E94D5490E9409210E94D9205092D60B7B
:103B60006092D70B7092D80B8092D90BE0C00E9464
:103B700009215090D60B6090D70B7090D80B809095
:103B8000D90B13EC29EC31E00E94E820E0F400911D
:103B9000E80406FD18C001FF16C00091EA0B05FD00
:103BA00029C000E414E601D41C3568F40E94092100
:103BB0000E94D9205092D60B6092D70B7092D80BEE
:103BC0008092D90BB4C000E21091EA0B12FD08E01C
:103BD000009335030FE50E94D5490E9409210E94F8
:103BE000D9205092D60B6092D70B7092D80B80924E
:103BF000D90B9DC010E21093350302FF98C007EC6B
:103C00000E94D54901E00093DF02A0923503A09203
:103C1000C00B00912A03077F00932A03A092EA0BAE
:103C2000A0920C047727F89482C00091E80406FD66
:103C30002AC00091E90407FF26C00091EA0B02FDAB
:103C400022C010E400E20E94D5211A30E0F40E9464
:103C500009215090D60B6090D70B7090D80B8090B4
:103C6000D90B1CE12EE43EE00E94E82008F45FC07E
:103C70000091F50B00FD06C001E00093F50B0AEE84
:103C80000E94D54954C008E0009335030E940921E1
:103C90000E94D9205092D60B6092D70B7092D80B0D
:103CA0008092D90B44C00091E80406FD0CC001FFCE
:103CB0000AC00091EA0B05FD2AC000E414E675D3A2
:103CC000183008F034C000E1009335030E94D92E6B
:103CD000009325030091EA0B0093520321E0209307
:103CE000F30B0AEA0093190301E00093DF02A092AC
:103CF0003503A092C00B00912A03077F00932A038B
:103D0000A092EA0BA0920C047727F89410C00E94AE
:103D100009215090D60B6090D70B7090D80B8090F3
:103D2000D90B13EC29EC31E00E94E82060F60895ED
:103D300058E00091ED0403FD51E004FD50E20E94C3
:103D40006D1F01B3052B01BB0E946D1F0E946D1FEB
:103D5000509501B3052301BB0E946D1F08955524A2
:103D6000422F493018F053944850FBCF66240894F2
:103D7000661C4A95E9F708951091DE02103009F4A7
:103D800029C00E94C109752F1091E60B103009F46B
:103D900021C071BB0E94C109752F0E946D1F770F52
:103DA000709308010E948E1F0E948E1F0E948E1F1A
:103DB0000E948E1FA1BA0E946D1FA092080101E00F
:103DC0000093DF02A092350321E02093F30B0AEA6F
:103DD00000931903A092DE020895009161021091F0
:103DE00062022091DD0B3091DE0B0217130731F0D8
:103DF0000091D20300FF02C00E94CE000091610238
:103E000010916202209127033091280302171307B3
:103E100008F448C00091360307FD44C00091CF0369
:103E200000FD0E944B0C0091CF0300FD3BC0A0920F
:103E300052030E94F5010000103009F421C00091E6
:103E40006702012B00936702009131030061009328
:103E50003103EEE9F0EA0E94340100916702112774
:103E6000ACE6B4E00E948001ECE6F4E00E944C0174
:103E7000A092DE0201E00093DF02A0920D0412C0C6
:103E800004E00093DF02A0923503A0920504E2D182
:103E9000C0D18FD15092A9026092AA027092AB0257
:103EA0008092AC020895B5D184D15092A50260925F
:103EB000A6027092A7028092A8029DD1AAD150902A
:103EC000A5026090A6027090A7028090A80210E45C
:103ED0002FE030E07DD188F308950091E70200FDE6
:103EE00019C097D166D15092A5026092A602709235
:103EF000A7028092A8027FD18CD15090A502609039
:103F0000A6027090A7028090A80210E126E030E09F
:103F10005FD188F30895E1DFE0DF08950091E702C3
:103F200000FD19C076D145D15092A5026092A6023B
:103F30007092A7028092A8025ED16BD15090A50228
:103F40006090A6027090A7028090A80214E82EE16B
:103F500030E03ED188F30895603021F0DFDF6A95CC
:103F600009F0FCCF0895E50DFA1D20810895FBDFCF
:103F7000262920830895E0933703F09338030091B6
:103F800026030A95E0EFF6E0E00FFA1D0081102FFE
:103F9000137031F00A950083E02E037009F002C01F
:103FA0000E94ED03309126033A9510E622E0130FAC
:103FB0002A1D0E2DF999FECF0E94C403E09137030C
:103FC000F0913803089510918102202F209512233B
:103FD00010938102109150041160109350040895C1
:103FE000A0924103009181020F7009F471C02090EA
:103FF00061023090620203FD05C002FD1DC001FD9B
:1040000035C04EC06AE026163A04B0F022279CD094
:1040100000918502003081F0201608F0202E2092B9
:10402000DA03022D003108F00FE00093CB0308E023
:104030000093410314E147C065E026163A04B0F04E
:10404000222782D000918402003081F0201608F0EF
:10405000202E2092D903022D003108F00FE00093AA
:10406000CB0304E00093410312E12DC062E0261669
:104070003A04B0F0222768D000918302003081F02A
:10408000201608F0202E2092D803022D003108F0CF
:104090000FE00093CB0302E00093410311E113C052
:1040A000009182020030A1F0201608F0202E20920C
:1040B000D703022D003108F00FE00093CB0301E09D
:1040C0000093410310E11093CE0302E00093CF036D
:1040D0000895A0924303A092410320906102309082
:1040E00062026091870222271091810214FF2BC087
:1040F000603009F428C026163A0428F125D011248E
:1041000000916802003071F4109181021F7E1093BB
:104110008102109150041160109350040027009305
:10412000410311C0021528F4201A269E500C1A1CB7
:10413000202E20924303252C312C2227009141036D
:104140000061009341030895623090F06624442496
:104150005524522C26163A042A0540F0639409F49B
:104160004394261A3A082A09A2F75524262C342CFF
:104170000895442720FD439521FD439522FD439555
:1041800023FD439524FD439525FD4395089555242E
:10419000662477248824089501911191219130811A
:1041A0000E0D1F1D2A1D3A1D308322931293029378
:1041B00008955090A1026090A2027090A302809096
:1041C000A40208958894111F221F331F001F089511
:1041D00000E01090A1022090A2023090A302409033
:1041E000A402F0DF510E621E731E801E15142604F9
:1041F000370448040895002E0091E70200FD07C02F
:10420000B090130308EC0A95F1F7BA94D9F7002D92
:10421000089506B51091A102011B10F0B9F419C060
:104220001091A202139581F42091A302239551F4D9
:104230003091A402339521F40DD033272227112782
:104240003093A4022093A3021093A20206B5009318
:10425000A1020895E0933703F0933803E1EAF2E016
:1042600014E306D0A6BCE0913703F091380308951B
:10427000A1921A95E9F7089515E01093DF02EEE791
:10428000F0EA0E9434010E944C01089531E000518F
:104290001742E8F7005F184D3FEE305F085E1340AD
:1042A000E0F708511C4F339504561040E0F70C59C5
:1042B00020EF205F0A50E8F7065F200F0895009175
:1042C000C9000E7F0093C90008950091C9000160E4
:1042D0000093C9000895242420925B030895509010
:1042E000BD026090BE027090BF028090C00218E1D3
:1042F00027EB30E00E94E82008F416C00E949501E8
:10430000A092A403A0927603A0923503A092DE02AD
:1043100001E012D07EDF4DDF5092B5026092B6020E
:104320007092B7028092B8020895E0E6F4E0E0935C
:104330004503F093460308950093DF0200E10093E4
:104340003A0300EA00934703A092DE02A0924403DE
:10435000A0922903A0922A03A0922C03A0920D04FC
:1043600008959924B9B0B02209F093941A95D1F721
:10437000192D08959924B0B0B02209F093941A959C
:10438000D1F7192D08959924B3B0B02209F0939470
:104390001A95D1F7192D08959924BCB0B02209F0CF
:1043A00093941A95D1F7192D08959924B09000018E
:1043B000B02209F093941A95C9F7192D08959924FC
:1043C000B2B2B02209F093941A95D1F7192D08953D
:1043D0009924B6B0B02209F093941A95D1F7192D0B
:1043E00008959924B0900601B02209F093941A958B
:1043F000C9F7192D089500913B0300FD31C00091CC
:10440000EA0B0E7F0093EA0B00E814E6BCDF1830DD
:1044100038F001E000933B0301B3046001BB12C01C
:1044200001E000933B0301B3046001BB0E948E1FB7
:1044300000E814E6A8DF1C3528F40091EA0B0160BF
:104440000093EA0B0E9409210E94D9205092D60BBA
:104450006092D70B7092D80B8092D90B002725C0A1
:104460000E9409215090D60B6090D70B7090D80B0A
:104470008090D90B1EE027E237E010919F02209137
:10448000A00233270E94E82060F400271091EA0B75
:1044900010FD0BC000E814E676DF183010F000279E
:1044A00004C001B30B7F01BB01E008950091EC044F
:1044B00003FF57C00091E80406FD53C01091CE0BD6
:1044C00010FD4FC00091120C00FD33C0009130016F
:1044D00007FF47C0009136011091110C153539F4D2
:1044E0000093D6030093130CA092110C3AC0103520
:1044F00069F40F3031F411E01093120CA092110CFA
:1045000030C00093100CA092110C2BC0003571F03C
:10451000053549F01091CE0B10FF02C00093110C2D
:10452000A092110C1EC00093110C1BC00093110C23
:1045300018C01091300115FF14C001FD09C00BEA2D
:10454000009336010091120C02600093120C09C016
:104550000091100C00933601A092120C006B0E9487
:10456000770A08950E94092181E00091E80406FD80
:1045700073C19CDF882700910F0C003009F46CC1D7
:1045800000FD60C101FD40C102FDC1C003FD49C085
:1045900004FD3CC005FD04C0A0920F0C81E05CC18D
:1045A0000091300105FF58C100911D0C00933601A8
:1045B0000E94770A04E000930F0C03EA00931D0C9D
:1045C0000E94D9205092C5026092C6027092C70222
:1045D0008092C8020091130C0435A1F0063591F0C9
:1045E00004E000930F0C0E94D9205092C502609203
:1045F000C6027092C7028092C802009136010091F3
:1046000036012AC1A092100C81E026C10091300130
:1046100005FF22C10AEA0093360100E200930F0C65
:104620001BC10091D603003009F4CEC00E94770A66
:104630006091D603A092D6030091D303013AF9F515
:104640006935C1F400911C0C00FD06C088270E944A
:104650009A3F01E000931C0C0E94D9205092C502A1
:104660006092C6027092C7028092C80200E1009375
:104670000F0CF2C0613589F401E00093100C0E9428
:10468000D9205092C5026092C6027092C7028092F1
:10469000C80204E000930F0CDFC0673549F40091B5
:1046A00067020160009367028395A092100CD4C04A
:1046B000643509F089C000E100930F0CCDC062356C
:1046C00089F407E00093100C0E94D9205092C50293
:1046D0006092C6027092C7028092C80204E0009302
:1046E0000F0CBAC0663521F400E100930F0CB4C082
:1046F000683501F783950091100C0D3028F4009176
:104700006702016000936702A092100CA5C010918F
:10471000CE0B10FF47C00091300107FF55C000913C
:1047200036011091D3031C3A19F40E94770A2CC069
:104730001B3A31F50E94770A0E94D9205092C50297
:104740006092C6027092C7028092C8020E9409213C
:104750005090C5026090C6027090C7028090C80257
:1047600014E82EE130E00E94E82008F00DC000912E
:10477000300107FFEBCF009136010E94770A04C099
:10478000053511F50E94770A0E94D9205092C50282
:104790006092C6027092C7028092C80208E000933D
:1047A0000F0C5AC00091110C003009F40DC010918B
:1047B00067021E7F10936702053531F40E94770A65
:1047C00008E000930F0C48C05090C5026090C602EC
:1047D0007090C7028090C8021AE522E632E00E947B
:1047E000E82088F0009167020160009367028395DA
:1047F000A092D603A092100C0091CE0B00FF03C034
:1048000008E00E94770A28C00091300105FF24C00B
:104810000091D303009336010E94770A04E00093CD
:104820000F0CA092D6030E94D9205092C50260922C
:10483000C6027092C7028092C802009136010091B0
:1048400036010AC00091300105FF06C00AEA009354
:10485000360102E000930F0C089588270091E804C8
:1048600006FDA3C200910F0C003009F49EC2A09275
:1048700098030E940921A092150300910F0C0A953C
:1048800009F459C20A9509F436C20A9509F408C216
:104890000A9509F4E0C10A9509F4C7C10A9509F41B
:1048A000A0C10A9509F479C10A9509F454C10A9581
:1048B00009F429C10A9509F489C00A9509F442C08E
:1048C0000091300105FFFCCF0CEA009336010E94F5
:1048D000770A0091300105FFFCCF01E0009336011B
:1048E0000E94770A00913601009136010E94092149
:1048F0000E94D9205092C5026092C6027092C702EF
:104900008092C8020E9409215090C5026090C602A0
:104910007090C7028090C80213EC29EC31E00E942D
:10492000E82008F03FC20091300107FFEBCF009173
:104930003601033529F00A3521F00C3519F734C258
:10494000E1CF2EC20091300105FFFCCF0BEA0093AE
:1049500036010E94770A0091300105FFFCCF01E08B
:10496000009336010E94770A0091360100913601CA
:104970000E9409210E94D9205092C5026092C6026D
:104980007092C7028092C8020E9409215090C5020D
:104990006090C6027090C7028090C80213EC29ECA8
:1049A00031E00E94E82008F0FDC10091300107FFCE
:1049B000EBCF00913601033529F00A3521F00C3593
:1049C00019F7F2C1E1CF0E94770AEAC10E940921DA
:1049D0005090C5026090C6027090C7028090C802D5
:1049E00013EC29EC31E00E94E82008F0DBC10091D3
:1049F000300107FFEBCF00913601083529F009356A
:104A000029F10C3519F7D0C10E9409215090C50237
:104A10006090C6027090C7028090C80213EC29EC27
:104A200031E00E94E82008F0BDC10091300107FF8D
:104A3000EBCF009136010F3138F70093750C006809
:104A40000E94770A06E000930F0C96C184E00E9452
:104A50009A3F0091300105FFFCCF0BEA009336012D
:104A60000E94770A0091300105FFFCCF02E000931D
:104A700036010E94770A00913601009136010E94AA
:104A800009210E94D9205092C5026092C6027092FC
:104A9000C7028092C8020E9409215090C50260900E
:104AA000C6027090C7028090C80213EC29EC31E076
:104AB0000E94E82008F076C10091300107FFEBCF9B
:104AC00000913601053519F00C3529F76DC10E94AA
:104AD00009215090C5026090C6027090C702809074
:104AE000C80213EC29EC31E00E94E82008F05AC11A
:104AF0000091300107FFEBCF00913601073039F705
:104B00000E94770A4DC10E9409215090C502609011
:104B1000C6027090C7028090C80210EF2AEF32E000
:104B20000E94E82008F03EC10091300107FFEBCF62
:104B300000913601053559F0053051F00C3321F460
:104B400006E000930F0C18C10C35E9F62DC1DBCF40
:104B50000E94770A11C10E9409215090C5026090FD
:104B6000C6027090C7028090C8021AE522E632E0C1
:104B70000E94E82008F016C10091300107FFEBCF3A
:104B800000913601053529F0043021F00C3519F774
:104B90000BC1E1CF0E94770AEFC00E94092150901B
:104BA000C5026090C6027090C7028090C8021AE5E4
:104BB00022E632E00E94E82008F0F4C000913001C3
:104BC00007FFEBCF00913601053539F0033031F0A6
:104BD000083011F00C3509F7E7C0DFCF0E94770AE3
:104BE000CBC00E9409215090C5026090C60270900F
:104BF000C7028090C80218E127EB30E00E94E8204D
:104C000008F0D0C00091300107FFEBCF00913601D2
:104C1000053539F0023031F00B3511F00C3509F75C
:104C2000C3C0DFCF0E94770AA7C00091300105FF03
:104C3000FCCF0AEA009336010A950E94770A009198
:104C4000300105FFFCCF01E00093360100913601F1
:104C50000091360191C00E9409215090C5026090D8
:104C6000C6027090C7028090C80218E127EB30E0BE
:104C70000E94E82008F096C00091300107FFEBCFBA
:104C800000913601063529F0013021F00B3519F776
:104C90008BC0E1CF0E94770A88270E949A3F6CC0A0
:104CA0000E9409215090C5026090C6027090C70210
:104CB0008090C80218E127EB30E00E94E82008F05D
:104CC00071C00091300107FFEBCF0091360105352F
:104CD00029F0013021F00C3519F766C0E1CF0E94B0
:104CE000770A15E00091980300FD10930F0C01E086
:104CF0000093980341C00E9409215090C502609022
:104D0000C6027090C7028090C80214E82EE130E01D
:104D10000E94E82008F046C00091300107FFEBCF69
:104D200000913601053519F00A3511F0E4CFE3CFD3
:104D30000E94770A21C00091300105FFFCCF0DEAE7
:104D4000009336010E94770A0091300105FFFCCFE5
:104D50000091740C009336010E94770A0091300193
:104D600005FFFCCF0091730C009336010E94770A77
:104D700000913601009136010E9409210E94D9203C
:104D80005092C5026092C6027092C7028092C80219
:104D900000910F0C039500930F0C0D3008F469CDB2
:104DA000882703C081E001C082E008958827009130
:104DB000E80406FD82C100910F0C003009F47DC1AA
:104DC0000E94092100910F0C0A9509F43CC10A9533
:104DD00009F418C10A9509F4D0C00A9509F4ABC0CA
:104DE0000A9509F483C00A9509F46BC00A9509F481
:104DF00045C00A9509F402C088275FC100913001BF
:104E000005FFFCCF0CEB009336010E94770A00915E
:104E1000300105FFFCCF01E0009336010E94770AC4
:104E20000091300105FFFCCF02E0009336010E94A3
:104E3000770A00913601009136010E9409215090B5
:104E4000C5026090C6027090C7028090C80218E147
:104E500027EB30E00E94E82008F02CC100913001DF
:104E600007FFEBCF00913601053529F00A3521F017
:104E70000C3519F721C1E1CF88271FC10E940921F4
:104E80005090C5026090C6027090C7028090C80220
:104E900013EC29EC31E00E94E82008F00BC10091EE
:104EA000300107FFEBCF00913601033529F00A35B9
:104EB00021F00C3519F700C1E1CF0E94770A88274D
:104EC000FCC00091300105FFFCCF0BEA00933601D6
:104ED0000E94770A0091300105FFFCCF01E00093AA
:104EE00036010091360100913601CEC00E940921A1
:104EF0005090C5026090C6027090C7028090C802B0
:104F000013EC29EC31E00E94E82008F0D3C00091B6
:104F1000300107FFEBCF00913601053539F0023043
:104F200031F00C3511F00D3509F7C6C0DFCF0E9406
:104F3000770A8827C2C00E9409215090C50260905C
:104F4000C6027090C7028090C80213EC29EC31E0D1
:104F50000E94E82008F0AEC00091300107FFEBCFBF
:104F600000913601063529F0013021F00C3519F792
:104F7000A3C0E1CF0E94770A87C00091300105FFEE
:104F8000FCCF0CEA009336010E94770A00913001B1
:104F900005FFFCCF00914B0412E0010F0093360196
:104FA0000E9409210E94D9205092C5026092C60237
:104FB0007092C7028092C8020091360100913601BA
:104FC0000E9409215090C5026090C6027090C702ED
:104FD0008090C80213EC29EC31E00E94E82008F030
:104FE00069C00091300107FFEBCF00913601053514
:104FF00029F0013021F00C3519F75EC0E1CF0E9495
:10500000770A42C00E9409215090C5026090C602F2
:105010007090C7028090C80213EC29EC31E00E9426
:10502000E82008F047C00091300107FFEBCF009166
:105030003601053519F00A3511F0E4CFE3CF0E94AF
:10504000770A88273AC00091300105FFFCCF0FEBAB
:10505000009336010E94770A0091300105FFFCCFD2
:105060000091780C009336010E94770A009130017C
:1050700005FFFCCF0091770C009336010E94770A60
:1050800000913601009136010E9409210E94D92029
:105090005092C5026092C6027092C7028092C80206
:1050A00000910F0C039500930F0C0D3008F488CE7F
:1050B000882703C081E001C082E008951127009194
:1050C000DE02003009F460C02091C403201708F408
:1050D0005BC0E0933703F0933803A0922703A092BC
:1050E0002803E0EFF7E00091DE020A95000FE00FE1
:1050F000FA1D019100932703208120932803022B9E
:1051000009F43EC0A0922603A09203041127209127
:10511000DE02E0E4F8E0019107FD03C00F7302171F
:1051200029F013951832B8F311272AC0139510935C
:1051300003041A95212E3324222764E00E94A42020
:105140002394209201042A9402E1029D102D05E08F
:10515000059D100D25E0052D033009F423E03327CC
:10516000E0EFF6E0E10FFA1D13950191037029F4C9
:1051700033952A95D1F711273327130F1093260360
:10518000E0913703F091380308950091E70200FDA4
:1051900019C00E9409210E94D9205092D20B60921E
:1051A000D30B7092D40B8092D50B0E9409215090A2
:1051B000D20B6090D30B7090D40B8090D50B0E94D3
:1051C000E82098F3089500913503003009F4BDC13B
:1051D00000FD72C101FD29C102FDE3C003FDADC0A8
:1051E00004FD73C005FD33C006FD04C007FDA09299
:1051F0003503ABC10E9409215090D60B6090D70BAC
:105200007090D80B8090D90B14E82EE130E010910B
:105210000502209106020E94E82008F068C100E221
:1052200012E3B1D8153008F090C101B30E7F01BB75
:105230000E946D1F009108010E7F0093080102E09B
:105240000093DF0200E2009335030C94CF1B0E9411
:1052500009215090D60B6090D70B7090D80B80909E
:10526000D90B14E82EE130E01091050220910602DE
:105270000E94E82008F03BC100E112E384D8153019
:1052800008F063C101B30E7F01BB51E01091EB0345
:1052900022270E94F43F0091080101600093080159
:1052A0000E946D1F01B3016001BB00E40093350350
:1052B0000E9409210E94D9205092D60B6092D70BF0
:1052C0007092D80B8092D90B40C10E940921509056
:1052D000D60B6090D70B7090D80B8090D90B14E848
:1052E0002EE130E010910702209108020E94E82090
:1052F00008F0FDC000E112E358D8153008F025C1D0
:1053000001B30B7F01BB55271091E3032091E40308
:105310000E94F43F01B3016001BB00E2009335033A
:105320000E9409210E94D9205092D60B6092D70B7F
:105330007092D80B8092D90B08C10E94092150901D
:10534000D60B6090D70B7090D80B8090D90B14E8D7
:105350002EE130E01091CD022091CE023091CF02AB
:105360000E94E82008F4F1C0009108010B7F00932F
:1053700008010E946D1F01B30F7B01BB01B30460E4
:1053800001BB00E1009335030E9409210E94D9204E
:105390005092D60B6092D70B7092D80B8092D90B9B
:1053A000D4C00E9409215090D60B6090D70B70900A
:1053B000D80B8090D90B14E82EE130E01091070251
:1053C000209108020E94E82008F091C000E212E358
:1053D0000E94D521153008F0B8C001B30B7F01BB86
:1053E0000E946D1F009108010E7F009308010E942A
:1053F000AF3124E83EE11091C10B0E94C70A20930F
:10540000CD023093CE024093CF0208E000933503E3
:105410000E9409210E94D9205092D60B6092D70B8E
:105420007092D80B8092D90B90C00E9409215090A5
:10543000D60B6090D70B7090D80B8090D90B14E8E6
:105440002EE130E010910502209106020E94E82032
:1054500008F04DC000E212E30E94C321153008F0AD
:1054600074C001B30E7F01BB0E946D1F0091080143
:105470000E7F0093080151E01091E3032091E403B3
:105480000E94F43F009108010160009308010E940E
:105490006D1F01B3046001BB04E0009335030E945B
:1054A00009210E94D9205092D60B6092D70B70929E
:1054B000D80B8092D90B49C00E9409215090D60B7D
:1054C0006090D70B7090D80B8090D90B14E82EE128
:1054D00030E010910502209106020E94E82038F485
:1054E00000E112E30E94C321153068F02EC0A1BA7A
:1054F000A09208010AEC0E94770A05E00093DF02FF
:10550000A092350322C001B30E7F01BB5527109135
:10551000EB0322270E94F43F0091080101600093F1
:1055200008010E946D1F01B3016001BB02E00093FE
:1055300035030E9409210E94D9205092D60B609217
:10554000D70B7092D80B8092D90B0895009130013F
:1055500005FFFCCF05E5009336010091300105FF02
:10556000FCCF05EA0093360108950091300105FF54
:10557000FCCF05E5009336010091300105FFFCCF1B
:105580000AE500933601089588270091CF0B00FDAE
:1055900026C099279093710301B30F7B01BB0027AD
:1055A0000E949B0D9A3509F013C001B3006401BB42
:1055B00002E00E949B0D01E010E20E94B121153033
:1055C00070F09091710393959093710391FFE4CFE4
:1055D0000CEC0E94770A05E00093DF0281E0089559
:1055E00088270091CF0B00FD85C000270E943E0D4B
:1055F0009A3561F00091DF020E30B1F390932303EE
:1056000001E00E943E0D9091230319C088270E945B
:105610009A3F01E00E943E0D9A3509F010C0002724
:105620000E949B0D9A3501F10091DF020E30E1F2EC
:105630009093230302E00E949B0D90912303092F76
:105640000E94770A0091DF020E3071F200912A0366
:10565000077F00932A0301E00093DF02A092350345
:10566000A092C00B81E046C001B3006401BB02E020
:105670000E949B0D9A3521F001B30F7B01BBDFCF58
:1056800000270E943E0D9A3561F00091DF020E3036
:1056900089F19093230301E00E943E0D9091230332
:1056A000EBCF84E00E949A3F01E00E943E0D9A35C4
:1056B00009F0E2CF04E00E949B0D9A3559F09093D7
:1056C000230301B30F7B01BB02E00E949B0D90916D
:1056D0002303B5CF01B30F7B01BB02E00E949B0DFA
:1056E0009A3501F088270091740C00FF03C081E017
:1056F0000E94D30C08950091E70400FF01C0DED69C
:1057000000912A0301FD47C30091C00007FF43C376
:10571000009167020F77009367020091C600009323
:10572000C60B0A3A41F41091ED0410FD04C005E5E2
:105730000E94770A30C30530F1F4A092CE0BA092FC
:10574000620301E01091EC0410FD0AE00093DF0217
:1057500000E100933A030AE50E94770AA092C00B89
:105760001AC3A092C00B01E00093130300EC022BBC
:105770000E94770A10C32091EE0426FF03C00E9406
:105780009C4E09C32091ED0420FF03C00E94974E58
:1057900002C32091EE0420FF03C00E94974EFBC27B
:1057A0002091ED0425FF18C00F700093DE02112731
:1057B00002E0009313030E94FB201A9511F421E0EC
:1057C000D0CF0091C00007FFF3CF0091C600009337
:1057D000E60B0E94BC1EDFC2102F107E103209F0B3
:1057E000FBC00F710093C00B1127222702E000932A
:1057F00013030E94FB201A9509F4B3CF0091C00057
:1058000007FFF4CF0091C6000093C10B2395112729
:1058100002E0009313030E94FB201A9509F4A1CF24
:105820000091C00007FFF4CF0091C6000093C20BA7
:105830002395112702E0009313030E94FB201A9581
:1058400009F48FCF0091C00007FFF4CF0091C6008C
:105850000093C30B2395112702E0009313030E94CA
:10586000FB201A9551F20091C00007FFF5CF00917F
:10587000C6000093C40B2395112702E00093130385
:105880000E94FB201A9509F4B8CF0091C00007FFD1
:10589000F4CF0091C6000093C50B77272224332450
:1058A000442488242091C20B0091C30B2F73022B38
:1058B00089F07160322E209334041091C30B212E95
:1058C000109333040E948F3F1093C80B2093C90B91
:1058D0003093CA0B2091C40B0091C50B122F107E80
:1058E000169516951695169516951093210C2F71F1
:1058F000022B89F07460822E20932E041091C50B28
:10590000412E10932D040E948F3F1093CB0B2093B8
:10591000CC0B3093CD0B0091ED0401FF11C0309101
:10592000C00B2091C10B2F701EE10E94C70AA092EC
:10593000370C2093380C3093390C40933A0C3AC012
:105940000091ED0403FF00C00091E90402FF32C0A2
:105950002091C00B0091C10B2F70022B59F10091C7
:10596000CE0B00FD0CC00091CF0B00FF08C02091B2
:105970008E022093C00B00918D020093C10B009109
:10598000CE0B00FD72601091C10B0E948F3F1093EF
:10599000350420933604022F012B61F40091CE0BC5
:1059A0001091CF0B012B31F402EA0E94770AA092EA
:1059B000C00BF1C11091C20B107C442717FD44604D
:1059C00016FD41601091C00B107114FD4260709380
:1059D000220C40930C0421C1103009F048C007701C
:1059E000013071F40FEF08B95F9A0091080101705E
:1059F00000930801A1BA0E946D1FA0920801ABCECE
:105A0000033039F40091CF0B21E002270093CF0B34
:105A1000A2CE023039F4A1BA0091080101700093BE
:105A2000080199CE043031F4C4D10E94770AA092C3
:105A3000C00BB1C1063059F411E02091EB0423FDF5
:105A400010E400910801012B0093080184CE073077
:105A500059F41EEF2091EB0423FD1FEB0091080188
:105A600001230093080177CEA092C00B94C1103699
:105A700009F06EC004FF19C00F7091F062E17AE77F
:105A800002FD80E401FD80E13091ED0431FD8AD317
:105A90003091ED0432FD37D23091EB0437FD33D233
:105AA0003091ED0432FF57CE76C1202F04EA2F70DB
:105AB00019F12A3031F5442731E6E0933703F093AA
:105AC0003803E0E7F8E00E941A2F00EA5030A1F016
:105AD000442730E610E02227E0933703F0933803A1
:105AE000E0E7F8E00E940F2FE0933703F0933803CC
:105AF000E0E7F8E072D12FCE0E94770AA092C00BA7
:105B00004AC1213059F410E0222730E64427E0E66C
:105B1000F4E00E94450330E6AED13DC1223059F495
:105B200010E014E030E64427E0E6F4E00E9445038C
:105B300030E6A1D130C1293009F70091C00005FF3E
:105B4000FCCF01E00093C60026C1A092C00B23C188
:105B5000103809F061C00F71003138F410910B0159
:105B6000107F102B10930B0116C1003131F40091FE
:105B700008010260009308010EC1013131F4009167
:105B800008010D7F0093080106C12091ED042871E2
:105B900089F423E9200F2A3A09F423952093D303AB
:105BA00021E020930F0C0E94B22220910F0C23FFC2
:105BB000FACFF1C00093D30324E020930F0C0E948E
:105BC00009210E94D9205092C5026092C6027092AB
:105BD000C7028092C80220913601209136010E94AE
:105BE00009215090C5026090C6027090C702809053
:105BF000C80211EE25EF34E00E94E82040F40E9434
:105C0000103920910F0C22FFEACF05EA01C008E508
:105C10000E94770AC0C0BFC0BEC00091E8040170F6
:105C2000E9F00091210C00FD19C00E944D4A20307E
:105C300081F00CEA0E94770A0091CF0B00FD09C0A9
:105C40000091CE0B00FD05C077278827A092C00BDE
:105C5000A2C00091E80400FD0E948F430AE50E9463
:105C6000770A0091200C00FF0BC00091210C02FF6D
:105C700007C040910C0440FF03C083E00E945840DD
:105C80007091220C70FD429872FD45980E946D1F24
:105C90000E94CB3E70FD0E94403D72FD0E94C63DB9
:105CA0003327442770FD0E94523E72FD0E948B3EB6
:105CB00070FD3093710072FD40936F0003E070FD42
:105CC0000093910072FD009381000E9409210E94BF
:105CD000D9205092D60B6092D70B7092D80B80923D
:105CE000D90B5092DA046092DB047092DC0480924B
:105CF000DD045092DE046092DF047092E004809232
:105D0000E1045092E2046092E3047092E404809211
:105D1000E5040091E9040073E1F0002770FD00E262
:105D200072FD00610DBBA0920C0CA0920D0CA09214
:105D3000000CA092010CA092FE0BA092FF0BA0926F
:105D4000160CA092170CA092140CA092150CA09205
:105D5000FD0B7894703029F00E9409210E94AE3921
:105D6000F9CFF8940091200C00FF15C00091210C90
:105D700002FF11C040910C0440FD0DC084E00E9460
:105D800058400E946D1F0E946D1F08B1046208B93F
:105D90000BE50E94770AA092C00B089503B1007F23
:105DA0000695069506950695109100011077012B32
:105DB000089503B1007F06950695069510910001A0
:105DC0001077110F012B1091000113FD016010914C
:105DD000EC0410FD0E94914E0895A0932303B0930C
:105DE0002403A0E6B2E031E401910D933A95E1F786
:105DF000A3EEB3E03EE001910D933A95E1F7A1E007
:105E0000B2E03DE001910D933A95E1F7A0912303B3
:105E1000B0912403E0913703F09138030895019184
:105E20000E94E50331504A09D1F7E0913703F09120
:105E300038030895CC2455270E94103800271030CD
:105E400099F00091C6000193C02631504A09A1F78C
:105E50000E94103851E00C2D103031F00091C60036
:105E60000C1511F451E002C00E94770AE09137034B
:105E7000F09138030895E0934503F093460311270A
:105E8000E0E6F4E00091C00005FFFCCF0191009333
:105E9000C60010273A95B1F70091C00005FFFCCF6E
:105EA0001093C600E0914503F091460308950F70EA
:105EB000D9F0093038F4102F0E94C10901B3052B25
:105EC00001BB12C01091EB0413FF04C00D3010F0A1
:105ED00069D20AC0102F17500E94C1090091080111
:105EE000052B0F7700930801089500934803009154
:105EF00008010160009308010E946D1F0E946D1F40
:105F00000091480308950F7009F44BC18827A092AF
:105F10003903093008F0DAC000933B03033000F581
:105F20001091EE04167321F00A950E943E0D39C1BE
:105F300080E31091EE0411FD80E1602F61FDD5DF5B
:105F400061FD80E251E05093E70B01B3052B01BBEB
:105F5000609105027091060261FF0E946D1F25C0CD
:105F60000730C0F48827033089F0043059F0602FDF
:105F7000002761FD02E00E949B0D092F0E94770A15
:105F800010C153C081E00E94D30C0BC182E00E947B
:105F9000D30C07C1093008F004C1882703FDA5DF31
:105FA0000E94981EA0920801FCC00E9409210E9434
:105FB000D9205092D60B6092D70B7092D80B80925A
:105FC000D90B0E9409215090D60B6090D70B70908E
:105FD000D80B8090D90B14E82EE130E0162F272F34
:105FE0000E94E82008F064C010E22091EE0421FD38
:105FF0000BC060913B0300E161FF06C000E20E941C
:10600000D521153080F3DDCF00E221FD082F0E945D
:10601000C321153040F32091EE0421FDD2CF00E1E1
:106020000E94C3211530F8F2CCCF0E9409210E94B2
:10603000D9205092D60B6092D70B7092D80B8092D9
:10604000D90B9AE50091390300FD9CEC0E940921CF
:106050005090D60B6090D70B7090D80B8090D90BD6
:1060600014E82EE130E01091CA042091CB040E9484
:10607000E820F0F48091C103803019F387FD10C04F
:10608000082F10E20E94D521153090F000913903BD
:1060900000FFD7CF0E949A4E9AE581FD09C0D1CF6B
:1060A0008F77082F10E20E94CC21153008F0C9CF5D
:1060B0005091E70B509501B3052301BB0E946D1F62
:1060C000A0920801092F0E94770A6BC00A30C1F420
:1060D0000091080101700093080101B30F7B01BB1F
:1060E0000091E80B08B901B3007801BB0E946D1F55
:1060F000009108010E7F00930801A0924B0451C04B
:10610000093051F401B3006401BB0AE50E94770A2B
:1061100001E000934B0445C00C3021F44ADE0E949C
:10612000770A3FC00B30D1F4992701E010E20E94BA
:10613000B121153008F0916008E010E20E94CC21F6
:10614000153008F0926002E010E20E94B121153093
:1061500008F09460092F0E94770A23C00D30A1F443
:106160000091EE0402FF07C000914B0400FD03C044
:106170000E94A50E02C00E94020E092F0E94770AFB
:106180000EE00093DF020DC00E3039F401B30F7B37
:1061900001BB0AE50E94770A04C00F3011F40E9487
:1061A0008F4308950F7009F4D9C0093008F0A4C0D6
:1061B000033078F480E1602F61FD97DE61FD80E2BD
:1061C00051E001B3052B01BB6091050270910602FD
:1061D0003AC0073020F591E00330B1F0043089F087
:1061E00080E1602F61FD81DE61FD80E254E001B35A
:1061F000052B01BB0E946D1F609107027091080280
:1062000047C073DE88E0992788E052E001B3052B90
:1062100001BB6091090270910A023AC09FC0093027
:1062200008F09CC0882703FD60DE58E001B3052B11
:1062300001BB0E946D1F01B3077F01BB0E946D1F50
:10624000A09208018BC00E9409210E94D92050927F
:10625000D60B6092D70B7092D80B8092D90B0E940C
:1062600009215090D60B6090D70B7090D80B80907E
:10627000D90B14E82EE130E0162F272F0E94E820DA
:1062800090F5082F10E20E94C321153060F1E7CF8E
:106290000E9409210E94D9205092D60B6092D70B00
:1062A0007092D80B8092D90B0E9409215090D60B86
:1062B0006090D70B7090D80B8090D90B14E82EE12A
:1062C00030E0162F272F0E94E82068F4803061F319
:1062D000082F10E290FF0E94CC2190FD0E94D52152
:1062E000153008F0E1CF509501B3052301BB0E94A2
:1062F0006D1FA092080132C00A30B1F4009108016C
:106300000B7F009308010E946D1F01B30F7B01BB3F
:106310000091E80B08B9009108010E7F0093080175
:1063200001B3007801BB1AC0093011F418D016C0AF
:106330000C3021F43EDD0E94770A10C00B3009F4C6
:106340000DC00D3021F4A1E00E94B10607C00E304F
:1063500009F404C00F3011F40E948F43089500E245
:1063600010E20E94D521153008F01BC001B3006473
:1063700001BB0E946D1F0091080104600093080199
:106380000E946D1F41B3486041BB0E946D1F477F53
:1063900041BB0E946D1F406141BB0E946D1F4F7E3B
:1063A00041BB08950D3069F10E30C1F001B30260B8
:1063B00001BB0E946D1F01B3016001BB00E10093AE
:1063C00039030E9409210E94D9205092D60B609275
:1063D000D70B7092D80B8092D90B25C001B3016006
:1063E00001BB00E2009339030E9409210E94D920D9
:1063F0005092D60B6092D70B7092D80B8092D90B2B
:1064000012C001B3016001BB00E4009339030E9494
:1064100009210E94D9205092D60B6092D70B70921E
:10642000D80B8092D90B0E9409215090D60B609016
:10643000D70B7090D80B8090D90B14E82EE130E088
:10644000109105022091060233270E94E820A0F453
:106450000091E80402FFE7CF0091390304FD06C074
:1064600012E30E94D521153038F0DDCF12E30E94EF
:10647000C321153008F0D7CF01B30C7F01BB0895BD
:106480000895C0933703D0933803C0EFD6E010E6E9
:1064900022E038EC08810C7F026009930E94CA0355
:1064A0003A95C1F721E020933B03A0927603A09296
:1064B0007703C0913703D0913803089500913503D5
:1064C000003009F43AC400FD84C301FDDFC202FDBF
:1064D0004AC203FDB8C104FDEDC005FD03C0A09292
:1064E0003503C7C410913B0310FF03C0A0923B03C8
:1064F0002FD51091E0031030A9F5009176030830F4
:1065000009F018C011601093E003A09276034427AD
:1065100040930C040027ECD40E94800865E02AE533
:10652000F22E20E20E94710200FFA2C0E1D4A092EC
:10653000E0039EC0093009F06DC012601093E003C3
:10654000A09276030027D4D40E94800865E02AEA4E
:10655000F22E20EC0E94710200FF8AC0C9D4A092E2
:10656000E00386C011FD2BC040910C04009176031E
:10657000003009F47DC0073031F424E04227409315
:106580000C04B6D475C0053011F4426003C0063067
:10659000F1F74160409352030027AAD4A0927603FA
:1065A0002AEAF22E20E26091520360670E94710293
:1065B00000FF02C09DD45CC003E69AD459C012FD0E
:1065C00029C040910C0400917603003009F450C0BA
:1065D000073031F424E0422740930C0489D448C0AA
:1065E000053008F045C0440F402B406A40935203E9
:1065F00000277ED4A09276032AEAF22E20EC609146
:1066000052030E94710200FF02C072D431C003E63F
:106610006FD42EC00530A1F40E94692017E004FD5C
:1066200018E01093DF02A092350311E004FD1093EF
:106630003E030E948E080E948E1F0E948E1F19C466
:106640001091090410FD13C01091800310FF10C0B9
:106650000E9472080E94FB2011E010930904A0928E
:106660008003E2E5F3EA0E9434010E944C01E3D486
:10667000A09276031091620311FFFBC310910904ED
:1066800010FF04C00E948E08A0920904EEE5F1EA12
:106690000E9434010E944C01F9C20BC0A0928003F9
:1066A0000CE0E9E6F2E0A1920A95E9F701E0009337
:1066B0003B03DFC310913B0310FF39C0A0923B03A3
:1066C000EEEFF1EA0E943401A0938F03B0939003A0
:1066D000009181021127A3E6B4E00E948001E3E665
:1066E000F4E00E948A01009168021127ACE6B4E050
:1066F0000E948001ECE6F4E00E948A01009187028A
:106700001127A4E7B4E00E948001E4E7F4E00E94CE
:106710008A010091890210918A02ACE7B4E00E94DC
:106720008001ECE7F4E00E948A010E944C01009194
:10673000700321E01091800310FD02270093700385
:10674000A09280031091620311FF0AC0EEE3F1EA08
:106750000E94340105E3009363040E944C0196C239
:1067600010917603103009F46BC0143009F448C05E
:10677000133081F11230C1F0113059F510918102BE
:1067800000FD04C01F3F29F1139503C0103009F12B
:106790001A9510938102012F24E011E20E94E50373
:1067A00001E000933B034CC01091680200FD04C05F
:1067B0001F3F79F0139503C0103059F01A951093CC
:1067C0006802012F24E018E00E94E50301E0009335
:1067D0003B0336C01091870200FD04C01F3F81F1CA
:1067E000139503C0103061F11A9510938702012FA1
:1067F00004E017E20E94E50301E000933B0320C0A0
:106800001091890220918A023AE04FEF00FD06C004
:10681000163F2407A8F4130F2A1D05C0412F422B51
:1068200079F0131B2A091093890220938A02012F01
:10683000322F1BE20000032F000001E000933B0316
:10684000A092760316C310913B0310FF48C0A0929C
:106850003B03EEE1F2EA0E943401009190020093C2
:1068600063040091910200936404009192020093EA
:1068700065040091930200936604009194020093D2
:1068800067040091950200936804009196020093BA
:1068900069040091970200936A04009198020093A2
:1068A0006B040091990200936C0400919A0200938A
:1068B0006D04C0938F03D0939003C3E7D4E009ED38
:1068C00010913903123020F01A9529911A95E9F7A1
:1068D00008830E944C01C0918F03D09190030091D6
:1068E000700321E01091800310FD022700937003D4
:1068F000A09280031091620311FF0AC0EEE3F1EA57
:106900000E94340104E3009363040E944C01BEC161
:1069100010917603103011F11130A9F42091390350
:106920002A95E0E9F2E0E20FFA1D1081193308F030
:106930001FE213951083012F10E3120F000001E0F6
:1069400000933B030BC0009139030B3008F0002784
:1069500003950093390301E000933B03A092DE020C
:10696000A092760386C210913B0310FF48C0A0920C
:106970003B03EEEDF1EA0E94340101E30093600471
:10698000A0938F03B0939003009182021127A2E697
:10699000B4E00E946B01E2E6F4E002E300936504D8
:1069A0000AE300936604009183021127A7E6B4E08E
:1069B0000E946B01E7E6F4E005E3009370040AE34C
:1069C00000937104009184021127A2E7B4E00E94B1
:1069D0006B01E2E7F4E001E30093770400E3009346
:1069E00078040AE300937904009185021127AAE74D
:1069F000B4E00E948001EAE7F4E00E944C011091AB
:106A0000800310FF0EC034E0E2E8F2E012E2A1924F
:106A1000002700003A95D9F711E010933B03A092AC
:106A200080031091620310FF19C004E00093CF03AC
:106A300034E0E2E8F2E012E2019100003A95E1F779
:106A40000091DD0B1091DE0B009361021093620246
:106A500011E0000000916202000018C10091610283
:106A600010916202102B39F0A0926102A092620292
:106A700011E010933B031091CF0310FDFAC102E027
:106A80000093CD0311E01093CF03F3C110913B03AA
:106A900010FF52C0A0923B03C0EFD6E00091BB03B1
:106AA0000A95C00FDA1D099103700093DC03099168
:106AB00003700093DE03A092DD03A092DF03EEE9F2
:106AC000F1EA0E943401A0938F03B09390030091E8
:106AD000BB031127A3E6B4E00E948001E3E6F4E0E3
:106AE0000E948A010091DC031091DD03A8E6B4E066
:106AF0000E948001E8E6F4E00E948A010091BB0355
:106B000003951127A3E7B4E00E948001E3E7F4E0D6
:106B10000E948A010091DE031091DF03A8E7B4E030
:106B20000E948001E8E7F4E00E948A010E944C0183
:106B3000A0918F03B09190031091620311FF07C0E1
:106B4000EEE1F1EA0E9434010E944C019FC01091D5
:106B5000800310FF39C01091E00310FD17C01091A1
:106B60007603103089F11A3F11F48BDC2DC029EB2C
:106B7000121750F51093BB0321E020933B032093A1
:106B8000E003A0927603A09277031EC0A092E003D8
:106B900020917603C0EFD6E00091BB030A95C00FA9
:106BA000DA1D18811C7F212B2993302F022F10E62C
:106BB00022E0130F2A1D0E94CA0321E020933B0309
:106BC000A0927603A0927703A0928003A092620322
:106BD00050C110913B0310FF4FC0A0923B03C0EF88
:106BE000D7E00091BB030A95000FC00FDA1D099191
:106BF0000093DC0309910093DD0309910093DE0308
:106C000008810093DF03EEE7F1EA0E943401A093CC
:106C10008F03B09390030091BB031127A4E6B4E067
:106C20000E946B01E4E6F4E00091DC031091DD03C7
:106C3000A7E6B4E00E948001E7E6F4E00E948A0142
:106C40000091BB0303951127A4E7B4E00E946B01F8
:106C5000E4E7F4E00091DE031091DF03A7E7B4E07E
:106C60000E948001E7E7F4E00E948A010E944C0143
:106C7000A0918F03B09190031091620311FF0FC098
:106C8000EEEFF0EA0E9434010E944C01A092E00372
:106C9000A0926203A0928003A09235034EC010918F
:106CA000800310FF45C01091E00310FD15C0109146
:106CB00076031030E9F12091C40323951217C0F533
:106CC0001093BB0321E020933B032093E003A092A9
:106CD0007603A09277032CC0A092E0032091760364
:106CE00030917703432F422B09F4C3C047E2203190
:106CF000340710F02FE037E2C0EFD7E00091BB037C
:106D00000A95000FC00FDA1D29933883402F022FF8
:106D100010E623E0140F2A1D0E94CA03032F0E94CD
:106D2000CA0321E020933B03A0927603A09277034D
:106D3000A0928003A09262039CC00091790300306E
:106D400041F4A092620301E00093790300933903B8
:106D500090C01091620311FD19C010FD59C010912F
:106D6000800310FF86C0A0926203A0928003A092CD
:106D700070030093350300913503043018F411E0DB
:106D80001093BB0301E000933B0373C0A092620326
:106D900000917903000F0F7309F401E00093790368
:106DA00000FD2FC001FD24C002FD1DC003FD0FC06A
:106DB00004FD05C0EEE5F1EA0E94340126C0EEE3D1
:106DC000F1EA0E94340105E3009363041EC00091C0
:106DD000E60401FF4EC0EEE3F1EA0E94340104E351
:106DE0000093630412C0EEE3F1EA0E9434010DC087
:106DF0001091F00F10935003EEE1F1EA0E9434017C
:106E000004C0EEEFF0EA0E9434010E944C0131C050
:106E10000E94950101E01091EC0410FD0AE000933E
:106E2000DF02A0926203A0928003A0927003A0925E
:106E30003503A0927903A092DE02A0923B03A092B8
:106E4000BB03A0927603A0927703A092E00300E137
:106E500000933A03A0926702A092E202A092630319
:106E60000E946D1F0E946D1F0E946D1F0E946D1F6A
:106E700000C00895E32FF42F3081362B308308951E
:106E8000009162030030F9F401E00093DF02222751
:106E90001BEC3091C403330FE0EFF7E00E94450391
:106EA000A0922F0304E0009330030E946D1F0E9404
:106EB0006D1F0E94D9205092BD026092BE02709256
:106EC000BF028092C0020895009176031127A7E7C0
:106ED000B4E00E946B01E7E7F4E00091670211273C
:106EE000ACE7B4E00E948001ECE7F4E00E948A0184
:106EF000602FEEE7F2EA0E9434010091E003037094
:106F00001127A6E6B4E00E946B01E6E6F4E00091EA
:106F100076031127ACE6B4E00E948001ECE6F4E0D1
:106F20000E948A0100910C041127A4E7B4E00E949A
:106F30006B01E4E7F4E0062F1127ACE7B4E00E9410
:106F40008001ECE7F4E00E948A010E944C01089560
:106F5000EEE5F2EA0E943401C9E6D2E0E2E6F4E0AE
:106F600012D0C1E7D2E0EAE6F4E00DD0CDE6D2E0FF
:106F7000E2E7F4E008D0CBE9D2E0EAE7F4E003D0BE
:106F80000E944C0108950991199129911AD040E36A
:106F9000102F02950F70040F01931F70140F11939F
:106FA000032F02950F70040F01933F70340F31933C
:106FB000022F02950F70040F01932F70240F21935D
:106FC00008955FEF5395005412442F40D8F7005CAA
:106FD0001D4B204F4FEE405F005A16482140D8F716
:106FE000005619472E4F4395005117422040D8F7BD
:106FF000005F184D2F4F3FEE305F085E1340E0F703
:1070000008511C4F339504561040E0F70C5920EFFF
:10701000205F0A50E8F7065F200F042F152F089510
:1070200011270E94FB201A9529F00091C00007FF4C
:10703000F8CF00C008950091C00007FFDCC00091A8
:10704000C6001AEA0113D7C0EBDF05E5103079F06E
:107050000091C60000930B04402FE0933703F09398
:10706000380300910B04007F003A11F001E5BDC028
:10707000D7DF02E51030D9F35091C60050930A04CF
:107080004527E0E7F8E00E94103803E5103079F377
:107090000091C600019340275150A9F70E94103873
:1070A00004E5103021F306E51091C6001417F9F637
:1070B000A0934803B0934903E0E7F8E000910B0484
:1070C00011EA011314C0A0EFB6E030910A04019157
:1070D0000D933A95E1F710E622E030910A04A0EF13
:1070E000B6E00D910E94CA033A95D9F772C012EA30
:1070F000011314C0A0EFB4E030910A0401910D9384
:107100003A95E1F710E620E030910A04A0EFB4E0F0
:107110000D910E94CA033A95D9F75BC013EA011397
:1071200014C0A0EFB5E030910A0401910D933A9597
:10713000E1F710E621E030910A04A0EFB5E00D91EF
:107140000E94CA033A95D9F744C014EA011314C047
:10715000A0E4B8E030910A0401910D933A95E1F76B
:1071600010EB23E030910A04A0E4B8E00D910E94F6
:10717000CA033A95D9F72DC015EA011314C0A0EF40
:10718000B7E030910A0401910D933A95E1F710E6CA
:1071900023E030910A04A0EFB7E00D910E94CA03EA
:1071A0003A95D9F716C016EA011313C0A3EEB3E05F
:1071B00030910A0401910D933A95E1F711E420E032
:1071C00030910A04A3EEB3E00D910E94CA033A95F0
:1071D000D9F7E0913703F0913803A0914803B091BB
:1071E00049030AE50E94770A06C0E0913703F0914F
:1071F00038030E94770A089503E00093A1000FEF7F
:107200000093A50006EF0093E30B0093A40031E088
:1072100039BB3091720031603093720078940895D8
:107220000091E80406FD99C000910F0C00FD88C094
:1072300001FD78C003FD6AC004FD5AC002FF8DC085
:107240000091D3030F700A950A9589F10A9561F1AF
:107250000A9539F10A9511F10A95E9F00A95C1F0FC
:107260000A9599F00A9569F00A9551F00A9539F056
:107270000A9521F00A9509F070C06FC06EC06DC00C
:107280006CC008E000930F0C68C083E092E011C06E
:1072900083E091E00EC082E092E00BC082E091E0DA
:1072A00008C081E093E005C081E092E002C081E087
:1072B00091E00EEA3091300135FFFCCF00933601AA
:1072C0000E94770A082F3091300135FFFCCF0093E0
:1072D00036010E94770A092F3091300135FFFCCF2B
:1072E000009336010E94770A01E000930F0C35C02D
:1072F0003091C00037FF31C09091C6008091F103FA
:107300000EEA1091ED0413FD0FEAD4CF3091C000C6
:1073100037FF23C00091C6000093F10300E1009302
:107320000F0C1BC03091300137FF17C000913601A0
:107330000A3599F40E94770A04E000930F0C0DC0FF
:107340003091300137FF09C000913601053529F42D
:107350000E94770A02E000930F0C089570FF27C087
:107360000091210407FF23C000FF21C00E7F00937E
:10737000210431E000912404109125042091260479
:10738000030F1A1D2A1D0093240410932504209333
:107390002604309138044091390450913A0403177F
:1073A0001407250718F00E94FD3C01C076D029C0C3
:1073B00071FF27C000915C0C07FF23C000FF21C0B4
:1073C0000E7F00935C0C31E000915D0C10915E0C1F
:1073D00020915F0C030F1A1D2A1D00935D0C109362
:1073E0005E0C20935F0C3091600C4091610C5091C9
:1073F000620C03171407250718F00E94123D01C004
:10740000A2D172FF28C00091220407FF24C000FF10
:1074100022C00E7F0093220431E0009127041091D6
:10742000280420912904030F1A1D2A1D0093270404
:10743000109328042093290430913B0440913C048C
:1074400050913D0403171407250718F00E94E83CEB
:1074500023C0CED021C071FF1FC00091230407FFBD
:107460001BC000FF19C00E7F0093230431E0009180
:107470002A0410912B04030F1A1D00932A04109361
:107480002B0430913E0440913F040317140718F079
:107490000E94273D01C001D208954FEF3091F10BBA
:1074A00030FF4EEF4093810C309121043670303024
:1074B00009F46AC031FF0BC0309146044091470483
:1074C00050914804031714072507D8F009C03091DC
:1074D000400440914104031714072A0598F04BC05B
:1074E00000912104097F009321040E9409210E9438
:1074F000D9205092DA046092DB047092DC0480920E
:10750000DD0475C00E9409215090DA046090DB040C
:107510007090DC048090DD0418E023E030E00E94ED
:10752000E82008F464C041E04093F10B0091D704D7
:107530001091D5040117F8F403950093D704E09354
:10754000CF04F093D004F3EAE2E7E00FFA1D0590D0
:1075500000921D04E091CF04F091D0040E94092113
:107560000E94D9205092DA046092DB047092DC040D
:107570008092DD043CC0009121040B7F02600093E7
:107580002104A092D20433C00E9409215090DA0451
:107590006090DB047090DC048090DD0418E023E050
:1075A00030E00E94E82008F422C00091D704A01621
:1075B000F0F40A950093D704E093CF04F093D0043D
:1075C000F3EAE2E7E00FFA1D059000921D04E09156
:1075D000CF04F091D0040E9409210E94D92050923A
:1075E000DA046092DB047092DC048092DD0408957A
:1075F0004FEF3091F20B30FF4EEF4093800C309103
:1076000022043670303009F46AC031FF0BC030916B
:10761000490440914A045091CC04031714072507EC
:10762000D8F009C030914204409143040317140775
:107630002A0598F04BC000912204097F0093220490
:107640000E9409210E94D9205092E2046092E30432
:107650007092E4048092E50475C00E940921509064
:10766000E2046090E3047090E4048090E50418E084
:1076700023E030E00E94E82008F464C041E0409339
:10768000F20B0091D8041091D4040117F8F403957B
:107690000093D804E093CF04F093D004F3EAE2E738
:1076A000E00FFA1D059000921F04E091CF04F091C5
:1076B000D0040E9409210E94D9205092E2046092D5
:1076C000E3047092E4048092E5043CC0009122043B
:1076D0000B7F026000932204A092D30433C00E9467
:1076E00009215090E2046090E3047090E4048090DB
:1076F000E50418E023E030E00E94E82008F422C00E
:107700000091D804A016F0F40A950093D804E093F1
:10771000CF04F093D004F3EAE2E7E00FFA1D0590FE
:1077200000921F04E091CF04F091D0040E9409213F
:107730000E94D9205092E2046092E3047092E40423
:107740008092E50408954EEF30916E0C30FF409327
:10775000A50030915C0C3670303009F46AC031FFFE
:107760000BC03091650C4091660C5091670C03176B
:1077700014072507D8F009C03091630C4091640CC0
:10778000031714072A0598F04BC000915C0C097F81
:1077900000935C0C0E9409210E94D9205092DE04C3
:1077A0006092DF047092E0048092E10475C00E9450
:1077B00009215090DE046090DF047090E004809016
:1077C000E10410E32CE030E00E94E82008F464C0FB
:1077D00041E040936E0C00916D0C10916C0C011700
:1077E000F8F4039500936D0CE093CF04F093D0046C
:1077F000F3EAE2E7E00FFA1D059000925A0CE091DF
:10780000CF04F091D0040E9409210E94D920509207
:10781000DE046092DF047092E0048092E1043CC0D8
:1078200000915C0C0B7F026000935C0CA0926B0CCF
:1078300033C00E9409215090DE046090DF047090F4
:10784000E0048090E10418E023E030E00E94E820AA
:1078500008F422C000916D0CA016F0F40A95009374
:107860006D0CE093CF04F093D004F3EAE2E7E00F6D
:10787000FA1D059000925A0CE091CF04F091D004CB
:107880000E9409210E94D9205092DE046092DF04F8
:107890007092E0048092E1040895309123043670E0
:1078A000303009F461C031FF08C03091CD044091FF
:1078B000CE0403171407D0F008C03091440440915F
:1078C00045040317140798F048C000912304097F6A
:1078D000009323040E9409210E94D9205092DE04C3
:1078E0006092DF047092E0048092E10470C00E9414
:1078F00009215090DE046090DF047090E0048090D5
:10790000E10410E821E030E00E94E82008F45FC0C4
:107910000091D9041091D6040117F8F4039500934F
:10792000D904E093CF04F093D004F3EAE2E7E00F48
:10793000FA1D059000921D04E091CF04F091D0044F
:107940000E9409210E94D9205092DE046092DF0437
:107950007092E0048092E1043AC0009123040B7F0E
:1079600002600093230433C00E9409215090DE047A
:107970006090DF047090E0048090E10410E821E062
:1079800030E00E94E82008F422C00091D904A0163B
:10799000F0F40A950093D904E093CF04F093D00457
:1079A000F3EAE2E7E00FFA1D059000921D04E09172
:1079B000CF04F091D0040E9409210E94D920509256
:1079C000DE046092DF047092E0048092E104089586
:1079D00000916F000E7F00936F00A092810008B1AC
:1079E000006C08B901E00093220400912C0400937C
:1079F0001F047B7F7093EF0B0895009171000E7F41
:107A000000937100A092910008B1086108B901E0EB
:107A10000093210400912C0400931D047E7F709339
:107A2000EF0B0895009172000E7F00937200A092F8
:107A3000A10008B1036008B901E000935C0C00915B
:107A40002C0400935A0C7D7F7093EF0B08950091E6
:107A500071000E7F00937100A092910008B1036045
:107A600008B9A0922A04A0922B0401E000932304F9
:107A700000912C0400931D047D7F7093EF0B0895FB
:107A800070FF40C0A0922404A0922504A092260476
:107A900040910C0440FD43980E946D1F00913804F2
:107AA0001091390420913A0460910F0263950E946D
:107AB000A93E3093D5044093400450934104A092D2
:107AC000D704009138041091390420913A04041B22
:107AD000150B2A0900934604109347042093480489
:107AE0000E946D1F34E83093210444980E940921BC
:107AF0000E94D9205092DA046092DB047092DC0478
:107B00008092DD04089571FF40C0A0925D0CA092A8
:107B10005E0CA0925F0C40910C0440FD40980E94C6
:107B20006D1F0091600C1091610C2091620C6091AE
:107B30000F0263950E94A93E30936C0C4093630C36
:107B40005093640CA0926D0C0091600C1091610C2C
:107B50002091620C041B150B2A090093650C1093ED
:107B6000660C2093670C0E946D1F34E830935C0C08
:107B700041980E9409210E94D9205092DE0460920F
:107B8000DF047092E0048092E104089572FF40C027
:107B9000A0922704A0922804A092290440910C04EA
:107BA00042FD46980E946D1F00913B0410913C04D9
:107BB00020913D046091100263950E94A93E30938C
:107BC000D4044093420450934304A092D8040091FB
:107BD0003B0410913C0420913D04041B150B2A0921
:107BE0000093490410934A042093CC040E946D1F13
:107BF00034E83093220447980E9409210E94D9203A
:107C00005092E2046092E3047092E4048092E504EE
:107C1000089571FF46C0A0922A04A0922B044091BF
:107C20000C0441FD40980E946D1F2227192F0E94CD
:107C30008F3F0091350430913604010F321F0093BD
:107C40003E0430933F04132F222760911102639565
:107C50000E94A93E3093D6044093440450934504B7
:107C6000A092D90400913E0410913F04041B150B0F
:107C70000093CD041093CE040E946D1F3091230415
:107C80003E7F3468309323045F980E9409210E944C
:107C9000D9205092DE046092DF047092E00480925A
:107CA000E10408952FB7F894309171003E7F30932E
:107CB00071003FEF3093950030911E043093940093
:107CC00030912C0430931D0431E038BB30917100A9
:107CD00031602FBFA092F10B2EEF2093810C0895FD
:107CE0002FB7F894509172005E7F509372005FEF4F
:107CF0005093A50050915B0C5093A40050912C041C
:107D000050935A0C51E059BB5091720051602FBFF3
:107D1000A0926E0C08952FB7F89440916F004E7F9B
:107D200040936F004FEF40938500409120044093B3
:107D3000840040912C0440931F0441E046BB4091D5
:107D40006F0041602FBFA092F20B2EEF2093800CAA
:107D50000895332744275527889427951795079525
:107D6000E093CF04F093D004F3EAE4E9E30FFA1DC3
:107D7000361758F4059015903395400D511D401756
:107D80005107A206A8F3402F512F3A95E091CF0456
:107D9000F091D00408950091C80B1091C90B209167
:107DA000CA0B009338041093390420933A040091CD
:107DB000CB0B1091CC0B2091CD0B00933B04109377
:107DC0003C0420933D040091200C00FF0E94FB3EE8
:107DD0007093D00B66276093D10B0E942A215EE03E
:107DE0005093D90B5EE45093D70B5CE15093D60BC4
:107DF000A0923503089500910102109102020093B0
:107E0000710C1093720C3090C20B2090C30B201693
:107E1000310628F4A09237040219130907C021E0A3
:107E200020933704201A310A022D132D00933304B6
:107E3000109334043091DB0B009103021091040283
:107E400000936F0C1093700C8090C40B4090C50B86
:107E5000430E8A1C4016810640F440910C044F7D6D
:107E600040930C04041918090AC040910C044061A5
:107E7000406240930C04401A810A042D182D00938F
:107E80002D0410932E04089571FF48C0009135040D
:107E900010913604012B09F441C05F980E946D1FB8
:107EA0000E94093E0E94523E3093710003E000930D
:107EB000910008B3016008BB2FBF0E9409210E94F6
:107EC000D9205092DE046092DF047092E004809228
:107ED000E1047894703019F00E94AE39FBCF009124
:107EE0000C0401FF15C00D7F00930C04409A10E4B0
:107EF00008E00E94C3211A3058F00091E80402FF04
:107F000007C004EA0E94D5490091CF0B00FF80E230
:107F10000091CE0B00FF02C088275F9A0895332797
:107F20000091C70B003029F0110F221F331F0A9553
:107F3000D9F708951091DB0B103009F454C000916B
:107F40003B040093450300913C04009346030091D9
:107F50003D040093390322270E948F3F10933B0476
:107F600020933C0430933D04A092D404A092420498
:107F7000A0924304A092D8041093490420934A0489
:107F80003093CC04A0922704A0922804A092290444
:107F900074E082FD469882FF469A0E946D1F3091E0
:107FA00022043E7F326830932204479845980E940D
:107FB0006D1F0E948B3E40936F0003E00093810091
:107FC0002FBF7894703011F0C9D9FCCFF89400918C
:107FD000450300933B040091460300933C04009149
:107FE000390300933D040895022F012B003009F45A
:107FF0005EC0009103023091040250FD07C0011BD6
:10800000320B009303023093040206C0010F321FAB
:1080100000930302309304024091360C040F3A1D82
:108020000093030230930402009101023091020296
:10803000040F3A1D00930102309302020E948F3F09
:1080400010933B0420933C0430933D041093490467
:1080500010934A04A092CC0474E050FF46980E940A
:108060006D1FA092D404A0924204A0924304A09257
:10807000D804A0922704A0922804A0922904309149
:1080800022043E7F326830932204479845980E942C
:108090006D1F0E948B3E40936F0003E000938100B0
:1080A0002FBF7894703019F059D9FCCFF894089507
:1080B0000091EC0404FF71C080935F0481FF03C052
:1080C0004298459837DF00918D0210918E02012B66
:1080D000003009F462C00091380400934503009118
:1080E00039040093460300913A04009339038091C8
:1080F0005F0471E080FF439A80FD43980E946D1FEA
:10810000A092D504A0924004A0924104A092D7046A
:1081100010918D0220918E020091350C82FD100F7E
:1081200082FD2A1D0E948F3F10933804209339044A
:1081300030933A0410934604209347043093480444
:10814000A0922404A0922504A09226043091210438
:108150003E7F3468309321044498A4DD309371004D
:1081600003E00093910042980E946D1F7894703054
:1081700011F0F4D8FCCFF89480915F04846081FD05
:10818000D9DE009145030093380400914603009323
:1081900039040091390300933A0408951091E503DE
:1081A000103009F454C00091380400934503009145
:1081B00039040093460300913A040093390371E0B7
:1081C00080FF439A80FD43980E946D1FA092D504C2
:1081D000A0924004A0924104A092D7041091E5031C
:1081E00022270E948F3F1093380420933904309344
:1081F0003A04109346042093470430934804A09215
:108200002404A0922504A0922604309121043E7FEC
:10821000346830932104429845DD3093710003E0C7
:108220000093910042980E946D1F7894703011F075
:1082300095D8FCCFF8940091450300933804009141
:108240004603009339040091390300933A040895DA
:108250007093220C71E00091100200933E0C00918B
:1082600038040093450300913904009346030091BC
:108270003A040093390380FF439A80FD43980E949B
:108280006D1FA092D504A0924004A0924104A09238
:10829000D70418EC22270E948F3F109338042093B4
:1082A000390430933A0410934604209347043093E2
:1082B0004804A0922404A0922504A09226043091A0
:1082C00021043E7F3468309321044298EBDC3093E4
:1082D000710003E00093910042980E946D1F06EC2C
:1082E000009323037894703069F010E400EC0E944E
:1082F000C3211A3010F032D8F6CF0E94FD3C0CE5B5
:1083000000932303F8940FEF08B9009145030093FD
:108310003804009146030093390400913903009317
:108320003A047091220C00913E0C009310020895C3
:108330007093220C71E000910F0200933E0C0091AB
:1083400038040093450300913904009346030091DB
:108350003A04009339034398A092D504A0924004B4
:10836000A0924104A092D7040E946D1F18EC22270E
:108370000E948F3F109338042093390430933A04BD
:10838000109346042093470430934804A092240499
:10839000A0922504A0922604009121040E7F046877
:1083A000009321047FDC3093710071FD0E94703EC8
:1083B00071FD5093720003E00093910071FD0093F2
:1083C000A10042980E946D1F06EC0093230378944D
:1083D0008827703081F010E400E80E94C3211A3031
:1083E00010F40BDB839580FD03C00E94AE39F1CF02
:1083F0000CE500932303F8940FEF08B900914503AF
:108400000093380400914603009339040091390326
:1084100000933A047091220C00913E0C00930F02DD
:1084200008957093220C74E00091100200933E0CAA
:1084300000913B040093450300913C0400934603E4
:1084400000913D04009339034698A092D404A09271
:108450004204A0924304A092D804A0922704A092C0
:108460002804A0922904309122043E7F3268309380
:108470002204479845980E946D1F18EC22270E94FD
:108480008F3F10933B0420933C0430933D041093A2
:10849000490420934A043093CC040E948B3E4093BD
:1084A0006F0003E00093810006EC0093230388270C
:1084B0007894703091F010E400E40E94C3211A30E7
:1084C00010F486DA839580FD03C00E94AE39F1CFA7
:1084D0000E94E83C0CE500932303F8940FEF08B9E1
:1084E0000091450300933B040091460300933C0434
:1084F0000091390300933D047091220C00913E0CD1
:1085000000931002089570FD429871FD5F9872FD0E
:10851000459800000E946D1F70FD0E94403D71FD56
:108520000E94833D72FD0E94C63D3327442770FDA3
:108530000E94523E71FD0E94703E72FD0E948B3E71
:1085400070FD3093710071FD5093720072FD409385
:108550006F0003E070FD0093910071FD0093A10096
:1085600072FD009381002FBF0E9409210E94D92033
:108570005092DA046092DB047092DC048092DD0495
:108580005092DE046092DF047092E0048092E10475
:108590005092E2046092E3047092E4048092E50455
:1085A000089580E1476040930C0477271091010201
:1085B00020910202022F012B003071F071600E94A5
:1085C0008F3F0091350C100F2A1D3A1D109338046F
:1085D0002093390430933A0410910302209104024D
:1085E000309166020091EB0403FF03C0130F2A1DB4
:1085F00013C000910C0405FF04C04091360C140F09
:108600002A1D00913F0C00FF07C013172A0518F020
:10861000131B2A0901C016C0022F012B003091F054
:1086200074600E948F3F00274091ED0444FF009149
:10863000E90B100F2A1D3A1D10933B0420933C04B4
:1086400030933D04703009F402C00E948342A0922E
:10865000DA0BA0920504A0923503A092D00B0E94E1
:108660002A210091710C1091720C00930102109359
:10867000020200916F0C1091700C00930302109392
:1086800004020E9409210E94D9205092D60B6092C8
:10869000D70B7092D80B8092D90B5092DA0460926B
:1086A000DB047092DC048092DD045092DE04609260
:1086B000DF047092E0048092E1045092E204609240
:1086C000E3047092E4048092E5045092B90260924F
:1086D000BA027092BB028092BC020091E90400735E
:1086E000E1F0002770FD00E272FD00610DBBA09279
:1086F0000C0CA0920D0CA092000CA092010CA09268
:10870000FE0BA092FF0BA092160CA092170CA09249
:10871000140CA092150CA092FD0B0000089570930C
:10872000220C75E000910C0400933C0CA0920C0408
:1087300000910F0200933D0C0091100200933E0C3B
:1087400001E000930F02009310020FEF0093380432
:10875000A0923904A0923A0400933B04A0923C04F6
:10876000A0923D04D0DE78947030B9F00E94AE390A
:1087700072FF08C010E200E40E94C321153010F01F
:108780000E94E83C70FF08C010E200E80E94C3218C
:10879000153010F00E94FD3CE7CFF89400912404BE
:1087A0002CD00093350C10913A0314FF0E94770AE5
:1087B00000915D0C22D00093760C10913A0314FFC7
:1087C0000E94770A0091270418D00093360C10916C
:1087D0003A0314FF0E94770A00913C0C00930C04AA
:1087E00000913D0C00930F0200930F0200913E0C8C
:1087F000009310027091220C089506950695069537
:10880000089588270091E80406FD5BC08091E90483
:1088100070FF8F7D72FF8F7E807309F452C050907D
:10882000B9026090BA027090BB028090BC0210E462
:108830002FE330E00E94E82008F443C088270E941C
:10884000D9205092B9026092BA027092BB02809213
:10885000BC020091000106FF02C005FD02C0839525
:1088600030C00091E904007309F42BC004FF12C06A
:1088700072FF10C00091000C1091010C2091160C99
:108880003091170C2017310708F015C00093160C13
:108890001093170C0091E90405FF13C070FF11C07D
:1088A0000091FE0B1091FF0B2091140C3091150CD0
:1088B0002017310710F0839504C00093140C109317
:1088C000150C089588270091E80406FD65C0009105
:1088D0003A0305FF00C00091E90404FF5DC072FF88
:1088E0005BC000910C0C013008F01FC02090000C00
:1088F0003090010C21E0220E3A1C222765E00E94F4
:10890000A4200091C50B1091C40B1F7100931A0C89
:1089100010931B0C2092160C3092170C02151305A5
:1089200008F403C00219130931F40DB30A7E0DBB1C
:10893000A0920C0C31C0212F102F0E948F3F40912C
:1089400027045091280460912904411B520B630BAA
:108950004093270450932804609329048395009141
:108960000C0C039500930C0CA092000CA092010C2F
:1089700000913A0305FF10C000911A0C0E94770A7B
:1089800000911B0C0E94770A0091160C0E94770A36
:108990000091170C0E94770A089588270091E80437
:1089A00006FD61C00091E90405FF5DC070FF5BC07A
:1089B00000910D0C013008F01FC02090FE0B30908C
:1089C000FF0B21E0220E3A1C222765E00E94A42022
:1089D0000091C30B1091C20B1F730093180C1093DE
:1089E000190C2092140C3092150C0215130508F482
:1089F00003C00219130931F40DB3057D0DBBA0921C
:108A00000D0C31C0212F102F0E948F3F4091240464
:108A10005091250460912604411B520B630B409337
:108A200024045093250460932904839500910D0C30
:108A3000039500930D0CA092FE0BA092FF0B0091EA
:108A40003A0305FF10C00091180C0E94770A0091AC
:108A5000190C0E94770A0091140C0E94770A009169
:108A6000150C0E94770A089588270091E80406FDF6
:108A700046C08091E90470FF8F7D72FF8F7E807306
:108A800009F43DC0803009F437C00E94092150909C
:108A9000D60B6090D70B7090D80B8090D90B13E059
:108AA00020E030E00E94E82020F000E50E94D54957
:108AB00023C084FF0FC072FF0DC00091FD0B037037
:108AC000033041F401E51091FD0B12FD02E50E9417
:108AD000D5498F7E85FFD6CF70FFD4CF0091FD0B97
:108AE0000871083179F603E51091FD0B15FD04E5D9
:108AF0000E94D5498F7DC6CF0DB300730DBB08957D
:108B00000091020C649920C000FF10C05090D50263
:108B10006090D6027090D7028090D80216E928E9BA
:108B200030E00E94E82008F43AC03AC001E0009327
:108B3000020C0E94D9205092D5026092D602709207
:108B4000D7028092D8022BC00091020C00FF12C005
:108B50000E7F0093020C5090D5026090D602709068
:108B6000D7028090D80210E120E030E00E94E82097
:108B700088F415C05090D5026090D6027090D7024C
:108B80008090D80216E928E930E00E94E82008F435
:108B900006C0CBCF31E0030F1A1D2A1D00C0882765
:108BA00008958827103009F472C00CB1012309F030
:108BB00037C0003029F100FF2FC05090C9026090EB
:108BC000CA027090CB028090CC0214E82EE130E013
:108BD0000E94E82008F45BC000913103016000931B
:108BE000310302E004E0EDE6F2E0A1920A95E9F734
:108BF0001DE0002734E00E94DE033A95E1F747C00C
:108C000001E00E94D9205092C9026092CA0270927B
:108C1000CB028092CC023BC002FF39C002E037C0D9
:108C2000003009F434C000FF15C00091DF020E309F
:108C300071F45090C9026090CA027090CB0280908B
:108C4000CC0218E023E030E00E94E82008F41FC0C6
:108C500081E01DC001FF0CC00E94D9205092C902C2
:108C60006092CA027092CB028092CC0204E00FC0E4
:108C70005090C9026090CA027090CB028090CC02E2
:108C800014E82EE130E00E94E82008F400C00895C6
:108C900010912C03119F0091640410916504010F41
:108CA0000025006808950091670207FD7CC00091CF
:108CB0002A0301FD77C00091F30B00FF74C00AE0A6
:108CC00000932903A092F30B02E000932A03E0E64D
:108CD000F4E0E0934503F09346030AEA10912C0375
:108CE00020913A03122B019300911903012701935C
:108CF0000091670201270193119300912503012739
:108D000001930091610200937C030127019300917C
:108D1000620200937D0328E0020F01270193009176
:108D20005203003001F40193A092520300915303C7
:108D300007FF05C0102F1F771093530301C00027B2
:108D40001091DC0B10FF02C00091DF0BA092DF0B33
:108D500001930091E00B0F771091EB0415FD98DF64
:108D60000083A0924403009167020F7B0093670287
:108D70000091EA04097061F40091DF02073041F4C8
:108D8000A0927C03A0927D03A092DD0BA092DE0B4B
:108D90000E94D9205092D1026092D2027092D302E6
:108DA0008092D40201D008950091670207FD89C026
:108DB00000912903003009F413C01091C00015FF81
:108DC00080C00A9500932903E0914503F091460382
:108DD00001910093C600E0934503F093460371C0F0
:108DE00000912A03027009F46CC00091C00007FDD5
:108DF0000FC05090D1026090D2027090D302809048
:108E0000D4021CE82BE530E00E94E82088F559C028
:108E10000091C60010912C0320914703122B0117DB
:108E200009F0000010912C031395183008F0112759
:108E300010932C03A0925203A0922503A092190331
:108E4000709167027072709367020091EA04097072
:108E5000C1F0009161021091620220917C03309177
:108E60007D03021B130B009361021093620209C081
:108E70000091670200680093670201E00093F30B22
:108E800002C0A0922903A0922A03A092E30B0091B2
:108E9000DC0B00FF0AC010912903103031F402608E
:108EA0000093DC0B20EA0E948E080E9409210E9498
:108EB000D9205092D1026092D2027092D302809255
:108EC000D40208955090D1026090D2027090D302E3
:108ED0008090D40210E42FE030E00E94E82008F4F3
:108EE000ECC100912A0300FD13C00091DC0B01FFCF
:108EF00002C00E9472080091C00005FFDEC111E0AF
:108F000010932A0300912B03006D0093C600D5C176
:108F10000091C00007FD19C05090D1026090D202AC
:108F20007090D3028090D4021CE82BE530E00E94C0
:108F3000E82008F4C2C100911E0C03950F3F20F0F9
:108F4000009108010D7F0000A5C10091C6000093AB
:108F500039031091820C10FF33C1102F107E103294
:108F600009F06CC00093C00B1127222702E0009388
:108F700013030E94FB201A9509F454C00091C0000D
:108F800007FFF4CF0091C6000093C10B2395009119
:108F9000EB0402FD6AC10091ED0405FD5CC11127DF
:108FA0000E94FB201A95F1F10091C00007FFF8CF55
:108FB0000091C6000093C20B239511270E94FB204D
:108FC0001A9581F10091C00007FFF8CF0091C6000B
:108FD0000093C30B239511270E94FB201A9511F1D2
:108FE0000091C00007FFF8CF0091C6000093C40BAA
:108FF000239511270E94FB201A95A1F00091C00033
:1090000007FFF8CF0091C6000093C50B01E0009365
:10901000130300E10093240C0AEA0093DE02A092FD
:10902000E60B38C101E000931303A0922E03A09237
:10903000C00B00EC022B0E94770A2AC1103409F001
:1090400091C02091EE0426FF03C00E949D4EB3C044
:109050002091E40B20FD21C00093C20BA092E50BF0
:1090600011270E94FB2022271A95E1F20091C000EF
:1090700007FFF7CF0091C6000093C30B21E02093B8
:10908000E40B20EA20932503209167022F7E209392
:10909000670221E02093F30BFBC0A092E40B209128
:1090A000C20B021711F02227BDCF0093C00B11276E
:1090B0000E94FB201A95B9F30091C00007FFF8CF7A
:1090C0000091C600009342031091C00B412F137012
:1090D000109343032091C30B021709F001C017C07E
:1090E000A0922503209167022065209367020091DA
:1090F0004203009361020091430300936202A09235
:109100004203A092430321E02093F30BC1C020E867
:109110002093E50B4C71469546950091DC0B00FFC2
:1091200009C042FF07C0435008E00093DF02A0924D
:10913000350308C007E00093DF0201E000933E031F
:10914000A0923B03142F0E94C109509341030E9437
:10915000D9205092B5026092B6027092B702809206
:10916000B80296C0103061F12091ED0420FF1CC0C0
:10917000212F2078203881F4102F1F701093DE02E9
:109180000077069506950695069503950093E60BE0
:1091900008E000932A030FC010761036E9F7102F6D
:1091A0001F711093420C07C0103849F40F710093DF
:1091B000F00BA09235030AE50E94770A69C068C0E7
:1091C000702F787176957695769570932D038091B2
:1091D0002B0383707817C9F5A0921E0C80912B0386
:1091E0008395883001E018F088270093820C8093E3
:1091F0002B03709167027F7770936702077009F401
:1092000047C000932E031091EC0411FF35C00130CC
:1092100011F4889A3DC0033059F401B30E7F01BBAD
:109220000E946D1F009108010E7F0093080130C05D
:109230000230F1F7009108010160009308010E94DB
:109240006D1F01B3016001BB23C000916702006480
:10925000009367021DC00091C00B0F700093DE02E7
:109260000091C10B0093E60B13C00091C10B00935A
:10927000DE02A092E60B0CC00091ED0402FF30D09C
:109280000091ED0402FD1AD00091ED0400FD02C032
:10929000A0922E0300912A030E7F00932A03A0922E
:1092A00039030E9409210E94D9205092D102609274
:1092B000D2027092D3028092D402089500912E03BC
:1092C000003009F40CC0063039F0073009F007C04F
:1092D00001B30F7B01BB03C001B3006401BB089560
:1092E0000091ED0400FD60C000912E03013009F4EF
:1092F00050C00230F1F1043071F10330B9F00630A2
:1093000079F0073039F0053009F04CC00EB1086033
:109310000EB948C0009108010F7B0093080142C0BC
:10932000009108010064009308013CC00091E8042A
:1093300001FF38C0009108010160009308010E94FC
:109340006D1F0E94981EA0923B03009108010E7FA2
:109350000093080127C00091EC0400FF03C0A09215
:10936000350320C00091ED0404FF1CC00E94B52A03
:1093700019C00091EA0404FD04C00EB1077F0EB9C4
:1093800011C000E10093240C0DC000E20093240CF6
:1093900009C00091EA0404FDF8CF009108010260C1
:1093A00000930801A0922E0308951091F80B10303D
:1093B00081F01A9559F01A9531F00093FC0B14E0E6
:1093C0001093F80B0DC00093FB0B05C00093FA0B34
:1093D00002C00093F90B1091F80B13951093F80B42
:1093E00008950091FA0B0093F90B0091FB0B009389
:1093F000FA0B0091FC0B0093FB0B089500912A03DC
:109400000F7EF1F40091C00005FF1AC00091F80B27
:109410000030B1F01091F90B1093C6000A9500933B
:10942000F80B003009F0DDDF0E9409210E94D920ED
:109430005092D1026092D2027092D3028092D402F2
:10944000089500916702003009F426C00091E604F7
:1094500001FF04C00091530305FF1EC0A092310319
:10946000A09232030091EB0400FF16C01091C000DF
:1094700015FFFCCF009167020093C6001091C00059
:1094800015FFFCCF00910E0C10E3003009F4012F02
:109490000093C600A0920E0C089522270091E804C4
:1094A00006FD1AC00091E80400FF16C022271091A3
:1094B000ED0413FD00ED13FD09C010E400E80E9467
:1094C000C3211A3010F021E007C000E410E40E942C
:1094D000C3211A3008F022E0089522270091E80401
:1094E00006FD0BC00091E90407FF07C010E400E28D
:1094F0000E94D5211A3008F0216008950091E804F7
:1095000006FD17C010E408E00E94D5211A3060F073
:109510000091530305FD0DC000620093530301EA5F
:1095200000000E94D54905C0009153030F7D0093B0
:10953000530308950091E80406FD54C010E400E1CF
:109540000E94D5211A3040F50091530306FD4AC010
:109550000E94092150907B0C60907C0C70907D0CD7
:1095600080907E0C19E02DE330E00E94E82008F4A2
:1095700039C00091530300640093530302EA0E9430
:10958000D5490E94D92050927B0C60927C0C70923D
:109590007D0C80927E0C26C00091530306FF22C0F2
:1095A0000E94092150907B0C60907C0C70907D0C87
:1095B00080907E0C19E02DE330E00E94E82090F0CE
:1095C000009153030F7B0093530306EA0E94D54991
:1095D0000E94D92050927B0C60927C0C70927D0C82
:1095E00080927E0C089522270091E80406FD0BC0AE
:1095F0000091E80401FF07C010E400E40E94D521B7
:109600001A3008F0216008950E9409215090D60B6D
:109610006090D70B7090D80B8090D90B17E823E996
:1096200033E00E94E82010F052E008C0552710E413
:1096300000E40E94D5211A3008F0516008952227D5
:109640000091E80406FD0CC00091E80403FF08C087
:1096500010E408E00E94D5211A3010F0216000C00B
:10966000089522270091E80406FD0BC00091E8044C
:1096700004FF07C010E400E10E94C3211A3008F083
:10968000216008950091EC0406FF15C017E61093C1
:109690007C00A0927B0015EC10937A000E940921B7
:1096A0000E94D9205092B1026092B2027092B3022D
:1096B0008092B4028F9808950091EC0406FF33C0A5
:1096C0000E9409215090B1026090B2027090B302E2
:1096D0008090B4021AE522E632E00E94E82018F1F8
:1096E00000917A0006FD1FC000917900003258F405
:1096F000003148F000933B0305EA0E94D5490091F0
:109700003B030E94D54915EC10937A000E94092171
:109710000E94D9205092B1026092B2027092B302BC
:109720008092B402000008950091340C0030F1F0F2
:1097300000FF01C03AC001FF0AC00091330C0F7353
:109740000093320C04E00093340CAEBC2EC003FF37
:109750002CC000E10093340C01E50CBD10913B0CD2
:1097600000910B01012B00930B011FC00E940921E6
:109770005090B9026090BA027090BB028090BC0217
:1097800010E126E030E00E94E82078F001ED0CBD09
:1097900000910B01092300930B0106E00A95F1F7F4
:1097A0007894AEBC01E00093340C08950091330C22
:1097B0001091320C15FF13C01F710091330C889467
:1097C000001F111F88941795079588941795079582
:1097D0008894179507950093330C1093320C0895D5
:1097E00000914B0C003009F45DC000FD46C001FF44
:1097F00059C090914E0C0E94944B0E9409215090A8
:10980000B9026090BA027090BB028090BC021CE862
:109810002BE530E00E94E82080F000E10093340C5A
:1098200001E50CBD10913B0C00910B01012B009345
:109830000B01A092320CA092330C0091340C04FF67
:1098400031C00E94D64B0091330C1091320C009322
:10985000470C1093480C04E000934B0CA092340C7E
:109860000E9409210E94D9205092B9026092BA0246
:109870007092BB028092BC0215C09DEF90934E0C7B
:10988000A092340C02E000934B0C0E9409210E942C
:10989000D9205092B9026092BA027092BB028092B3
:1098A000BC02A7CF089500914B0C003019F401E0E1
:1098B00000934B0C95DF00914B0C02FFFBCF2091E6
:1098C000470C3091480C07EA7DD001E000934B0C27
:1098D000089500914C0C003009F45DC000FD46C0B5
:1098E00001FF59C090914E0C0E94944B0E94092197
:1098F0005090B9026090BA027090BB028090BC0296
:109900001CE82BE530E00E94E82080F000E10093A5
:10991000340C01E50CBD10913B0C00910B01012BA7
:1099200000930B01A092320CA092330C0091340CE6
:1099300004FF31C00E94D64B0091330C1091320CC1
:109940000093490C10934A0C04E000934C0CA09235
:10995000340C0E9409210E94D9205092B9026092D1
:10996000BA027092BB028092BC0215C097EF90932E
:109970004E0CA092340C02E000934C0C0E94092182
:109980000E94D9205092B9026092BA027092BB0232
:109990008092BC02A7CF089500914C0C003019F4BE
:1099A00001E000934C0C95DF00914C0C02FFFBCFC3
:1099B0002091490C30914A0C08EA04D001E0009350
:1099C0004C0C08951091C00015FFFCCF0093C60009
:1099D0001091C00015FFFCCF3093C6001091C0005D
:1099E00015FFFCCF2093C60008958091A30395999D
:1099F00033C080FF23C05090CD026090CE027090A3
:109A0000CF028090D00218E927E030E00E94E820E1
:109A100008F471C00EEC1091E60410FD0E94D549C7
:109A200010913103106110933103009108010D7FF3
:109A30001091EA0410FF009308015DC081608093DB
:109A4000A3030E94D9205092CD026092CE02709260
:109A5000CF028092D0024FC080FF24C08E7F8093BF
:109A6000A3035090CD026090CE027090CF02809000
:109A7000D00212E720E030E00E94E82008F43BC06A
:109A800080688093A3032091A2030E94864E0091D8
:109A9000E60400FD07C0E090A203FF240E94874E69
:109AA000A092BB0300912A0301FD25C087FF16C0C9
:109AB0005090CD026090CE027090CF028090D00284
:109AC00014E82EE130E00E94E820A8F08F7780644F
:109AD0008093A30321E02093F30B0DC086FF0BC0FE
:109AE00000912903003039F400912A03027019F41F
:109AF0008F7B8093A30308950091840C00FD1DC00B
:109B000000E20093C00BA092C10B00918F02000FE6
:109B1000E0EFF5E0E00FFA1D119120811093C20BE8
:109B20002093C30BE0EFF4E0E00FFA1D11912081C8
:109B30001093C40B2093C50B86C00091ED0402FF67
:109B400014C008E010E20E94B121153008F07BC07B
:109B500075E00091390300930C0476D0009139032D
:109B600015E00127009339035FC001FF02C0BBD09D
:109B70006AC001E010E20E94DF219927153010F43D
:109B8000BFCF0000929B44C0919B35C000B10095AF
:109B9000802F003009F457C010913B03102329F0A7
:109BA00011E0109308010E946D1F10913B031827CC
:109BB00010933B03082F00FD1CC001FD18C002FDDF
:109BC00014C003FD10C004FD0CC005FD08C006FD57
:109BD00004C007FF38C08F9A2EC08E9A2CC08D9A71
:109BE0002AC08C9A28C08B9A26C08A9A24C0899A47
:109BF00022C0889A20C074E00091390300930C04BD
:109C000023D00091390314E00127009339030CC0DD
:109C100071E00091390300930C0416D000913903D0
:109C200011E0012700933903703019F00E94AE391A
:109C3000FBCFF89408C063E00E94AC1FA1BA0E9459
:109C40006D1FA0920801089500918F02000FE0EFB0
:109C5000F5E0E00FFA1D219110810E948F3F1093D3
:109C600038042093390430933A04E0EFF4E0E00F35
:109C7000FA1D219110810E948F3F10933B04209385
:109C80003C0430933D040E9483420E9409210E94BB
:109C9000D9205092D60B6092D70B7092D80B80923D
:109CA000D90B5092DA046092DB047092DC0480924B
:109CB000DD045092DE046092DF047092E004809232
:109CC000E1045092E2046092E3047092E404809212
:109CD000E5045092B9026092BA027092BB0280927F
:109CE000BC027894089591E000E210E20E94DF2126
:109CF000153008F008C090930B010E948E1FA092AF
:109D00000B01990FC1F708950895089508950895D6
:109D1000089508950895089508950895089508955B
:109D2000089508950895089508950895089508954B
:109D300008950895089508950895089500800F03E3
:109D400000009A000000020800800F0300009A0043
:109D5000000004080100070300009C0100480C00FB
:109D600001000F0300009A000000841000800F0320
:109D700000009A00000000080100070300009C0199
:109D800000480C000100010000003000000001004C
:109D900001000500000008000000004001004F0322
:109DA00000C09A0000908020010043030000B4002E
:109DB00000208404810005030000900000181400B6
:109DC0000100000000004000000001000100050348
:109DD0000000B400002084028100450300009000D0
:109DE00000181400010045030000A8000010040042
:109DF00081000503000090000018540001000503D5
:109E00000000B400001084010100000000004000C8
:109E1000000000080100020000000000000028000F
:109E2000010005030000A8000010040081000503E4
:109E300010002C00002006000102050A0000415419
:109E4000453056302B434D47463D310D415445304A
:109E50000D00415456302B434D47463D310D415482
:109E60002B434D47533D22220D0005050A160600DF
:109E70000701010101004B30303E30000A000100B3
:109E80003000415445300D00415456300D004154CE
:109E90002B434D47463D310D41542B4346554E3DD6
:109EA000300D41542B434D47533D22383930333820
:109EB000333831373038220D30303130321A050E18
:109EC0000C060700080D02031F010F1011121314D6
:109ED000151617181900102030405060700020200F
:109EE00020202020202020202020202020204FBFA4
:109EF000BA61B72047534D2020202020202041B3B5
:109F0000BF6FBC61BF20B3BABBC6C065BD20BA700D
:109F10006567B8BF20202020207079B2202042C37E
:109F2000676165BF63C7204E202020202020BA70C3
:109F30006567B8BF20202020202020202020B76186
:109F4000B26570B8BF652020BF6FB361702020205C
:109F50002020202020202020202020202020A16F31
:109F6000BF6FB36F3A2063BE6163B8B26F20B76151
:109F700020BE6FBA79BEBA79202020202020486107
:109F8000B26570B8BF6520BD6FBC65702020BF6F23
:109F9000B361706120202020B8202A202020546F37
:109FA000B361704E20202020202020202020B76187
:109FB000BA6FBDC0B8BB63C72020202020204FBE91
:109FC000BB61BFB8BF65202020202020702E4367D2
:109FD00061C0B820676F202020202020207042C35D
:109FE0006761C0612063BF61BA61BD61202020202C
:109FF00020202020202020202020202020204861F8
:10A00000B6BCB8BF6520BABD6FBEBA79202022BBEE
:10A010006567222CB761BF65BC222A222020546FBD
:10A02000B361704E20202020202020202020676F48
:10A03000BEBB61BFB8BF65202020202070204FBE6E
:10A04000BB61C065BD6F203030303020702E2020C5
:10A05000B8B7203030303020702E202020204BBD6B
:10A060006FBEBA61202223222D636761C061B8BB35
:10A07000B8204E20BF6FB3617061202020204FBFF9
:10A08000BA61B720BA79BEC670BDB8BA6120636F35
:10A090006FB2E6B8BF65206FBE65702D70794FBF97
:10A0A000BA61B720B3C36761C0B820202020636FB6
:10A0B0006FB2E6B8BF65206FBE65702D70794FBF77
:10A0C000BA61B720BD61BBB8B36120202020B36F57
:10A0D000B7B37061BF206FBEBB61BFC320204F5DAF
:10A0E000B8B26FBA20BD65BF2020202020202020DC
:10A0F00020202020202020202020202020207065CB
:10A10000B6313AE565BD61202020202020202020A6
:10A1100020202020202020202020202020207065AA
:10A12000B6323ABA6FBBB8C06563BFB36F202020A8
:10A13000202020202020202020202020202070658A
:10A14000B6333ABE617061BC202020202020202040
:10A15000202020202020202020202020202070656A
:10A16000B6363A63C065BF20202020202020202062
:10A170002020202020202020202020202020E565D5
:10A18000BD6120203A202020207079B22020E56592
:10A19000BD6120203A202020207079B22020BA6FA3
:10A1A000BB202020203A2020202020202020BA6F11
:10A1B000BB202020203A2020202020202020BA6F01
:10A1C000BB20203A20202020202020202020BA6FF1
:10A1D000BB20203A20202020202020202020313A9F
:10A1E000202020202020202020202020202020206F
:10A1F00020202020202020202020202020206367D5
:10A200003A2020202020BA6FBB3A20202020BD6FAA
:10A21000BC3A2020202020BC203A2020202054E4DA
:10A220003A20202020202020202020202020202014
:10A2300020202020202020202020202020205065A9
:10A24000B62E20B26563BEBB61BFBDC3B9206367D4
:10A2500061C0613A20202020202020202020BA70D8
:10A260002020202020202C63202020202020BF2000
:10A270002020202020202CBD20202020202079BE3E
:10A280007020BE7031202020202020202020B7BD4B
:10A2900061BA2020202020202020202020204D6175
:10A2A0007274696E69204269616E636F476F6C6496
:10A2B0002020A86F63BF61B3C4BF652063BF61BACC
:10A2C00061BD42C3B26570B8BF65204D61727469EB
:10A2D0006E694269616E636F202020202020702EFD
:10A2E0002020476F6C642020202020202020702E0A
:10A2F00020205A206FBFC065BF20202020202020B2
:10A30000202020202020202020202020202020204D
:10A310002020636761C0B8202020202020BD65BFB9
:10A320002020BA79BEB8BF6520BF6FB3617020200E
:10A3300020204FBFBA61B72020636761C0B82020DA
:10A340002020636F6FB2E6B8BF65206FBE65702DC9
:10A350007079B761BEB863C46FBFA8BA202020204F
:10A3600020202020202020202020202020202020ED
:10A3700020200000003A60788A9BA4ACB4BABFC425
:10A38000C9CFD6DEE6EBEFF1F3F7C3CED6DEE6EBD0
:10A39000EFF1F3F73100620062007F009D00BA0028
:10A3A000D700FA0012002C004D006A008600A400BD
:10A3B0000101010101020202020204040404040476
:10A3C000040404040101010101010101010102026F
:10A3D000020202020202020204040404040404044D
:10A3E0000404010101010101010101010101010157
:10A3F0000101010101010202020202020202020243
:10A40000020202020202020202020202020202022C
:10A41000020202020202010402020201040202011B
:10A420000204010204010204020102040102040107
:10A4300002040201020401020401020402010204F6
:10A4400001020401020440081010204008101020EE
:10A45000400808081010102020204008080810109C
:10A46000102020204008080810101020202040084C
:10A470000808101010202020FFFFFFFFFFFFFFFF44
:10A48000FFFFFFFFFFFFFFFFFFFFFFFFFFFFFFFFDC
:10A49000FFFFFFFFFFFFFFFFFFFFFFFFFFFFFFFFCC
:10A4A000FFFFFFFFFFFFFFFFFFFFFFFFFFFFFFFFBC
:10A4B000FFFFFFFFFFFFFFFFFFFFFFFFFFFFFFFFAC
:020000023000CC
:00000001FF
